:100000000C943A0F0C9454120C944D0F0C944D0F09
:100010000C944D0F0C944D0F0C944D0F0C948E15A9
:100020000C944D0F0C944D0F0C944D0F0C946813C1
:100030000C944D0F0C944D0F0C94F3120C944D0F27
:100040000C944D0F0C944D0F0C949F140C944D0F69
:100050000C9478140C944D0F0C944D0F0C944D0F80
:100060000C944D0F0C944D0F4000005600014000C1
:10007000012A00010A0000040000080201810000BA
:100080005600004A616E1F4665621C4D61721F4139
:1000900070721E4D61791F4A756E1E4A756C1F4144
:1000A00075671F5365701E4F63741F4E6F761E4435
:1000B00065631F53756E646179004D6F6E6461797D
:1000C0000054756573646179005765646E65736487
:1000D000617900546875727364617900467269646D
:1000E000617900536174757264617900B300BA007C
:1000F000C100C900D300DC00E300000303060104D3
:100100000602050003059281E7D6B4A39200514090
:10011000362503625100205465726D696E616C0072
:10012000808386898C8F9295989C9FA2A5A8ABAE60
:10013000B0B3B6B9BCBFC1C4C7C9CCCED1D3D5D872
:10014000DADCDEE0E2E4E6E8EAECEDEFF0F2F3F52B
:10015000F6F7F8F9FAFBFCFCFDFEFEFFFFFFFFFFE0
:10016000FFFFFFFFFFFFFEFEFDFCFCFBFAF9F8F7C7
:10017000F6F5F3F2F0EFEDECEAE8E6E4E2E0DEDCDF
:10018000DAD8D5D3D1CECCC9C7C4C1BFBCB9B6B3F8
:10019000B0AEABA8A5A29F9C9895928F8C898683C0
:1001A000807C797673706D6A6763605D5A575451CD
:1001B0004F4C494643403E3B383633312E2C2A279C
:1001C0002523211F1D1B1917151312100F0D0C0AC3
:1001D00009080706050403030201010000000000EE
:1001E00000000000000001010203030405060708E7
:1001F000090A0C0D0F1012131517191B1D1F2123AF
:1002000025272A2C2E313336383B3E404346494C75
:100210004F5154575A5D6063676A6D707376797C8D
:100220004A6452000102040810204080420050003D
:100230004700303132333435363738394142434460
:1002400045460CF80C46F846F8F80CF8FF01FE019C
:1002500001FE01FEFE01FEFE010101FEFE01FE01A6
:1002600001FE01FEFEFF0B694F0B8C4FFF0B697FF8
:100270000B8C4FFF0B694F0B8C7FFF66026D027476
:10028000020B694F0B8C4F0BAF4FFF0B697F0B8C31
:100290004F0BAF4FFF0B694F0B8C7F0BAF4FFF0B1B
:1002A000697F0B8C7F0BAF4FFF0B694F0B8C4F0B94
:1002B000AF7FFF0B697F0B8C4F0BAF7FFF81028BF2
:1002C0000295029F02A902B3020B694F0B8C4F0BE0
:1002D000AF4F0BD24FFF0B697F0B8C4F0BAF4F0B08
:1002E000D24FFF0B694F0B8C7F0BAF4F0BD24FFFE1
:1002F0000B697F0B8C7F0BAF4F0BD24FFF0B694FFE
:100300000B8C4F0BAF7F0BD24FFF0B697F0B8C4FCA
:100310000BAF7F0BD24FFF0B694F0B8C7F0BAF7F67
:100320000BD24FFF0B697F0B8C7F0BAF7F0BD24F34
:10033000FF0B694F0B8C4F0BAF4F0BD27FFF0B693D
:100340007F0B8C4F0BAF4F0BD27FFFC902D602E35E
:1003500002F002FD020A031703240331033E030CDB
:100360000102030405060708090A0B0C0102030435
:1003700005060708090A0B0000010001010001FF42
:1003800001FF00FFFF00FF53657269616C20496E39
:10039000204F766572666C6F77200A0D004E6F7283
:1003A0006D616C0053686F72742053312020204DB2
:1003B000656E75004C6F6E672020533120202043FE
:1003C00068616E67650053686F7274205332202035
:1003D0002048656C70004C6F6E67202053322020DF
:1003E000205265626F6F74004368616E67652F4DC0
:1003F000656E7500533120202020202020202049C8
:100400006E6372656D656E7400533220202020206B
:1004100020202020416476616E636500526566721B
:100420006573683A00557054696D653A00DF0619C6
:10043000EBF406A9EB9D0355CDA4030AB8B4030A57
:10044000A3C6030A8ED6030A79E8033C5FF4030AC5
:100450004A09040A351C040A1925040A0400008EFE
:100460001900008E04434D564B006024402569243A
:10047000102685078B07820794074E4650554C423D
:10048000001A26122825284B255325562405050336
:1004900002030944544148494F5253574700442DE1
:1004A0008B2DF62DCB2BFB2CB42BE92BEF2B232CF8
:1004B0007C2F20415652204F7363696C6C6F7363BD
:1004C0006F706520436C6F636B2000312064696737
:1004D00069742076616C75652028302D00322064A7
:1004E0006967697420006872733A20006D696E73E1
:1004F0003A2000736563733A2000796561723A208F
:10050000006D6F6E74683A20006461793A20004390
:10051000616E63656C2F54696D656F7574004E6113
:100520006D65200028432932303130204A616E2029
:10053000646520526965000D0A00342068657820E2
:10054000646967697420494F43544C3A200044530E
:10055000542066697820002048656C703A0D0A4185
:100560003A204170706C69636174696F6E205365E5
:100570006C656374696F6E2028302E2E35290D0A44
:10058000423A204275726E2D696E207072657665F2
:100590006E74696F6E0D0A433A20416C61726D2072
:1005A0006F6E2F6F66660D0A443A204368616E676E
:1005B0006520446174650D0A463A20436C6F636B95
:1005C0002046616365204D6F64652028302E2E35EE
:1005D000290D0A473A2047505320496E7075740D13
:1005E0000A493A20494F43544C0D0A4B3A2043687C
:1005F000726F6E6F20446973706C61790D0A4C3AAA
:10060000204C454420626C696E6B696E670D0A4D23
:100610003A205050532054726967676572204D6FBD
:1006200064650D0A4E3A204E756D6572696320440B
:100630006973706C6179204D6F64652028302E2EAF
:1006400035290D0A503A20506C6179204D6F646550
:100650002028302E2E33290D0A523A205265736518
:100660007420454550726F6D20436F6E6669670D4B
:100670000A533A20446973706C6179205374617431
:1006800075730D0A543A204368616E67652054699A
:100690006D650D0A553A204368616E6765204453C5
:1006A00054206D6F64650D0A563A20566572626F6C
:1006B0007365204F75747075740D0A573A2043683E
:1006C000616E6765204E616D6500436F6D6D616E93
:1006D00064284820666F722068656C70293A00446F
:1006E0007574636874726F6E697800537061726BB1
:1006F00066756E0056342E306473000101010101ED
:1007000000010101010000010101000000010100E0
:1007100000000001000000000001000000000101D5
:100720000000000101010000010101010080FE80C4
:10073000F2008DFE8CF9009AFC99F700A6F8A5F45A
:1007400000B3F4B1EF00BFEEBAE500CAE6C7E200BD
:10075000D4DED0DA00DDD5D9D100E5CBE1C800ED9B
:10076000BFE4BA00F3B4EEB200F7A7F3A600FB9B18
:10077000F69A00FD8EF88D00FD80F18000FD73F883
:100780007400FB66F66700F75AF35B00F34DEE4F1B
:1007900000ED41E44600E536E13900DD2CD93000BA
:1007A000D423D02700CA1BC71F00BF13BA1C00B335
:1007B0000DB11200A609A50D009A05990A008D0336
:1007C0008C08007F037F0F007203730800650566C5
:1007D0000A0059095A0D004C0D4E12004113461CD7
:1007E00000351B381F002B232F2700222C2630001A
:1007F0001A361E390012421B47000C4D114F0008DB
:100800005A0C5B00046609670002730774000281DA
:100810000E8100028E078D00049B099A0008A70C28
:10082000A6000CB411B20012BF1BBA001ACB1EC82E
:100830000022D526D1002BDE2FDA0035E638E20083
:1008400040EE45E5004CF44EEF0059F85AF40065CF
:10085000FC66F70072FE73F9FF80FE80FD81FD816A
:10086000FC008DFE8DFD8EFD8EFC009AFC99FB9B9D
:10087000FB9AFA00A6F8A6F7A7F7A7F600B3F4B21A
:10088000F3B4F3B3F200BFEEBEEDC0EDBFEC00CAAF
:10089000E6C9E6CBE5CAE500D4DED3DDD5DDD4DCA0
:1008A00000DDD5DCD4DED4DDD300E5CBE5CAE6CA75
:1008B000E6C900EDBFECBFEEBEEDBE00F3B4F2B38F
:1008C000F4B3F3B200F7A7F6A7F8A6F7A600FB9BD0
:1008D000FA9AFC9AFB9900FD8EFC8EFE8DFD8D0030
:1008E000FD80FC80FE81FD8100FD73FC73FE74FDC4
:1008F0007400FB66FA67FC67FB6800F75AF65AF863
:100900005BF75B00F34DF24EF44EF34F00ED41EC1C
:1009100042EE42ED4300E536E537E637E63800DDE6
:100920002CDC2DDE2DDD2E00D423D324D524D4259C
:1009300000CA1BC91BCB1CCA1C00BF13BE14C014A9
:10094000BF1500B30DB20EB40EB30F00A609A60A70
:10095000A70AA70B009A0599069B069A07008D0324
:100960008D048E048E05007F037F048004800500C3
:1009700072037204730473050065056606660667F4
:1009800007005909590A5A0A5A0B004C0D4D0E4DD1
:100990000E4E0F00411341144214421500351B3610
:1009A0001B361C371C002B232C242C242D25002225
:1009B0002C232D232D242E001A361A371B371B38D3
:1009C000001242134213431443000C4D0D4E0D4EC2
:1009D0000E4F00085A095A095B0A5B000466056756
:1009E00005670668000273037303740474000281D0
:1009F00003810382048200028E038E038D048D0026
:100A0000049B059A059A06990008A709A709A60A52
:100A1000A6000CB40DB30DB30EB20012BF13BF137A
:100A2000BE14BE001ACB1ACA1BCA1BC90022D5238A
:100A3000D423D424D3002BDE2CDD2CDD2DDC00359B
:100A4000E636E636E537E50040EE41ED41ED42ECB5
:100A5000004CF44DF34DF34EF20059F859F75AF7A4
:100A60005AF60065FC66FB66FB67FA0072FE72FDD3
:100A700073FD73FCFF7AEB7AD90080E883EB89EB96
:100A80008CE88CE580D98CD900B5E4B5D20000D2D1
:100A9000BBD5BEDBBEDEBBDEB8D2ACDEAC0000E256
:100AA00086E589EB89EE86EE83EB80EE7DEE7AEBD0
:100AB00077E577E27A00E580EB8000E04CD44CDD0E
:100AC00055DD430000B831AC31AC28B528B825B8A5
:100AD00022B51FAF1FAC220000852182247C24791F
:100AE0002179157C12821285158518821B7C1B7951
:100AF000180047315331532E502B4D254D1F0022E6
:100B00004C1F4F1F52225528552B522B4F284C2239
:100B10004C1F491F46224328432B462B49284C0093
:100B2000001D841A811A81148111841187148A1A74
:100B30008A1D871D7B1A781478117B000021BE2145
:100B4000AC000027BB2ABE30BE33BB33AF30AC2A6B
:100B5000AC27AF27BB000049E449D2000053E4535F
:100B6000D2FF0073EF76F27CF27FEF7FEC73E07FD1
:100B7000E0008DE981E98AF28AE000AAE2AAD000C9
:100B800000B0DFB3E2B9E2BCDFBCDCB9D9BCD6BC93
:100B9000D3B9D0B3D0B0D300B3D9B9D900D0BCD079
:100BA000AA0000E2B3D6B3DFBCDFAA0000DC89DC18
:100BB0007700EE89E289E280EB80EE7DEE7AEB77DA
:100BC000E577E27A00D055D0430000E252DF55D9F4
:100BD00055D652D646D943DF43E246E249DF4CD9E7
:100BE0004CD6490000AA2DAA1B0000B02DBC2DBC7C
:100BF0002AB927B621B61B00007B217B0F00831882
:100C0000801B801E832189218C1E8C1B89188318D0
:100C100080158012830F890F8C128C15891800495A
:100C20002F491D00005B295826582652264F294F70
:100C30002C522F582F5B2C5B20581D521D4F20002B
:100C4000001E52215527552A522A4F1E432A43007F
:100C5000002F52325538553B523B46384332432FD2
:100C6000462F5200001187148A1A8A1D871D84118D
:100C7000781D780000238A237800001EBB21BE2740
:100C8000BE2ABB2AB81EAC2AAC00002FBB32BE382D
:100C9000BE3BBB3BB82FAC3BAC000040DD43E04962
:100CA000E04CDD4CDA40CE4CCE000051DD54E05A31
:100CB000E05DDD5DDA5AD75DD45DD15ACE54CE51B8
:100CC000D10054D75AD7FF76DF8ADF0079DF80F36F
:100CD0000079F380DF0083DF83F30087F387DF0091
:100CE00076F38AF300ADD1B5D100B1D1B1E500AD55
:100CF000E5B5E50000D2ABDEAB00D6ABD6BF00DA7F
:100D0000ABDABF00D2BFDEBF00DC76EE7600E07665
:100D1000E08A00E576E58A00EA76EA8A00DC8AEE77
:100D20008A00C942DF4200CE42CE5600D242D2569D
:100D300000D642D65600DA42DA5600C956DF5600CF
:100D400000A922B92200AD36B122B53600A936B9C4
:100D5000360000751489140079287D1481280085D7
:100D60001485280075288928004322592200463618
:100D70004A224E3600512251360055225536004344
:100D800036593600001D42394200225626422A5664
:100D9000002E422E5600324232560036423656005F
:100DA0001D5639560011772377001477148B0018DD
:100DB00077208B00188B207700118B238B00002469
:100DC000AB32AB0027AB2FBF0027BF2FAB0024BF38
:100DD00032BF0048D15AD1004BD153E5004BE55307
:100DE000D10056D156E50048E55AE5FF007AEB7A86
:100DF000D90080E883EB89EB8CE88CE580D98CD92D
:100E000000E286E589EB89EE86EE83EB80EE7DEEEF
:100E10007AEB77E577E27A00E580EB800085218246
:100E2000247C24792179157C1282128515851882FB
:100E30001B7C1B7918001D841A811A81148111846E
:100E40001187148A1A8A1D871D7B1A781478117BE2
:100E5000FF80EC8080FF8BEC8080FF96EA8080FF33
:100E6000A1E78080FFABE38080FFB6DE8080FFBF1C
:100E7000D88080FFC8D18080FFD0C98080FFD7C0D4
:100E80008080FFDDB68080FFE2AC8080FFE6A2803C
:100E900080FFE9978080FFEB8C8080FFEB80808073
:100EA000FFEB758080FFE96A8080FFE65F8080FF4E
:100EB000E2558080FFDD4A8080FFD7418080FFD0EF
:100EC000388080FFC8308080FFBF298080FFB62334
:100ED0008080FFAB1E8080FFA11A8080FF96178064
:100EE00080FF8B158080FF80158080FF74158080C7
:100EF000FF69178080FF5E1A8080FF541E8080FF8C
:100F00004A238080FF40298080FF37308080FF2F78
:100F1000388080FF28418080FF224B8080FF1D5554
:100F20008080FF195F8080FF166A8080FF147580C3
:100F300080FF14808080FF148C8080FF1697808053
:100F4000FF19A28080FF1DAC8080FF22B68080FF49
:100F500028C08080FF2FC98080FF37D18080FF406C
:100F6000D88080FF49DE8080FF54E38080FF5EE709
:100F70008080FF69EA8080FF74EC8080FF8280803F
:100F8000E67E808280FF81808AE67E818180FF818B
:100F90008095E47E818180FF81809FE27E818180D7
:100FA000FF8180A9DE7E818180FF817FB3D97E822F
:100FB000817FFF817FBBD37E82817FFF817FC4CC15
:100FC0007E82817FFF817FCBC57E82817FFF817F93
:100FD000D2BC7E82817FFF807FD8B37F82807FFFFB
:100FE000807FDDAA7F82807FFF807FE1A07F82807B
:100FF0007FFF807FE3967F82807FFF807FE58B7F0E
:1010000082807FFF7F7EE58080827F7EFF7F7FE51D
:101010007680827F7FFF7F7FE36B80827F7FFF7F91
:101020007FE16180827F7FFF7F7FDD5780827F7FCE
:10103000FF7E7FD84D81827E7FFF7E7FD245818279
:101040007E7FFF7E7FCB3C81827E7FFF7E7FC435AB
:1010500081827E7FFF7E7FBB2E81827E7FFF7E7FAF
:10106000B32881827E7FFF7E80A92381817E80FFDD
:101070007E809F1F81817E80FF7E80951D81817E85
:1010800080FF7E808A1B81817E80FF7E817F1B8224
:10109000807E81FF7E81751B81807E81FF7E816ADB
:1010A0001D81807E81FF7E81601F81807E81FF7E29
:1010B00081562381807E81FF7E814D2881807E81C3
:1010C000FF7E82442E817F7E82FF7E823B35817F40
:1010D0007E82FF7E82343C817F7E82FF7E822D4530
:1010E000817F7E82FF7F82274E807F7F82FF7F828B
:1010F0002257807F7F82FF7F821E61807F7F82FFF9
:101100007F821C6B807F7F82FF7F821A76807F7F49
:1011100082FF80821A817F7E8082FF80821A8B7F8D
:101120007F8082FF80821C967F7F8082FF80821E6C
:10113000A07F7F8082FF808222AA7F7F8082FF80C3
:101140008227B37F7F8082FF81822DBC7E7F818258
:10115000FF818234C57E7F8182FF81823BCC7E7F8E
:101160008182FF818244D37E7F8182FF81824CD93C
:101170007E7F8182FF818156DE7E808181FF818139
:1011800060E27E808181FF81816AE47E808181FFCF
:10119000818175E67E808181FF828080BC7E808235
:1011A00080FF818086BC7E818180FF81808CBB7EB8
:1011B000818180FF818092BA7E818180FF818098C9
:1011C000B77E818180FF817F9EB47E82817FFF8197
:1011D0007FA3B17E82817FFF817FA8AD7E82817FE8
:1011E000FF817FACA97E82817FFF817FB0A47E8258
:1011F000817FFF807FB39E7F82807FFF807FB69953
:101200007F82807FFF807FB9937F82807FFF807F96
:10121000BA8D7F82807FFF807FBB877F82807FFF48
:101220007F7EBB8080827F7EFF7F7FBB7A80827FD4
:101230007FFF7F7FBA7480827F7FFF7F7FB96E8060
:10124000827F7FFF7F7FB66880827F7FFF7E7FB354
:101250006281827E7FFF7E7FB05D81827E7FFF7EA6
:101260007FAC5881827E7FFF7E7FA85481827E7F03
:10127000FF7E7FA35081827E7FFF7E7F9E4D818295
:101280007E7FFF7E80984A81817E80FF7E809247AC
:1012900081817E80FF7E808C4681817E80FF7E8082
:1012A000864581817E80FF7E817F4582807E81FFB1
:1012B0007E81794581807E81FF7E81734681807E3B
:1012C00081FF7E816D4781807E81FF7E81674A81BB
:1012D000807E81FF7E81624D81807E81FF7E825C87
:1012E00050817F7E82FF7E825754817F7E82FF7E87
:1012F000825358817F7E82FF7E824F5D817F7E8216
:10130000FF7F824C63807F7F82FF7F824968807F7E
:101310007F82FF7F82466E807F7F82FF7F8245745F
:10132000807F7F82FF7F82447A807F7F82FF8082FE
:1013300044817F7E8082FF808244877F7F8082FF1E
:101340008082458D7F7F8082FF808246937F7F8071
:1013500082FF808249997F7F8082FF80824C9E7FBE
:101360007F8082FF81824FA47E7F8182FF818253B2
:10137000A97E7F8182FF818257AD7E7F8182FF813E
:10138000825CB17E7F8182FF818261B47E7F8182B7
:10139000FF818167B77E808181FF81816DBA7E8008
:1013A0008181FF818173BB7E808181FF818179BCD6
:1013B0007E808181FF05941994196C056C05940653
:1013C000951A951A6D066D0695FF0F6C0F94109483
:1013D000106CFF0594199419800580056C196C1A1E
:1013E0006D066D067F1A7F1A930693FF0594199474
:1013F000196C056C066D1A6D1A9506950005801816
:10140000800018810681FF059405801880001881EE
:101410000681069500196C19941A951A6DFF199496
:10142000059405801980196D066D056C196C001AFC
:101430006D1A81068106951A95FF0594056C196C45
:10144000198006800006811A811A6D066D0695FFC7
:1014500005941994196C1A6D1A950695FF0594193F
:1014600094196C056C059406951A951A6D066D060F
:101470009500068018800018810681FF056C196CA4
:101480001994059405801880001881068106951A24
:10149000951A6D066DFFB513CA13D313EC13071419
:1014A0001E143A1450145D147C14058406840685B9
:1014B000058500057C067C067B057B004C844D84FD
:1014C0004D854C85004C7C4D7C4D7B4C7BFF103812
:1014D0003810100010006C6C48000000000000285C
:1014E0007C28287C28002038403008701000646474
:1014F0000810204C4C00205050205448340030300C
:1015000020000000000010202020202010002010CB
:101510001010101020000028387C3828000000101F
:10152000107C10100000000000000060604000000F
:1015300000780000000000000000003030000004CF
:1015400008102040000038444C54644438001030E7
:101550001010101038003844041820407C00384423
:10156000043804443800081828487C0808007C40E7
:1015700040780444380018204078444438007C0403
:1015800008102020200038444438444438003844AF
:10159000443C04083000000060600060600000000F
:1015A00030300030302008102040201008000000AB
:1015B0007C00007C00002010080408102000384443
:1015C00004181000100038445C545C403800384463
:1015D00044447C444400784444784444780038448B
:1015E00040404044380078444444444478007C40BF
:1015F000407840407C007C40407840404000384487
:10160000405C44443C004444447C4444440038101E
:1016100010101010380004040404444438004448F6
:101620005060504844004040404040407C00446C82
:101630005444444444004464544C444444003844B6
:10164000444444443800784444784040400038449E
:10165000444454483400784444784844440038446E
:101660004038044438007C1010101010100044441E
:10167000444444443800444444444428100044440E
:1016800054545454280044442810284444004444EA
:1016900044281010100078081020404078003820AE
:1016A00020202020380000402010080400003808C6
:1016B0000808080838001028440000000000000056
:1016C0000000000000FC30301000000000000000AE
:1016D00038043C443C0040407844444478000000D6
:1016E00038444044380004043C4444443C00000076
:1016F000384478403800182020782020200000004E
:101700003C44443C0438404070484848480010007D
:101710001010101018000800180808084830404041
:1017200048506050480010101010101018000000B1
:101730006854544444000000704848484800000081
:101740003844444438000000784444447840000061
:101750003C4444443C040000582420207000000015
:10176000384038043800002078202028100000007D
:10177000484848582800000044444428100000000D
:101780004444547C28000000484830484800000089
:101790004848483810600000780830407800182029
:1017A00020602020180010101000101010003008C9
:1017B000080C080830002850000000000000387CA9
:1017C0007C7C7C7C3800596F7572204E616D652081
:1017D000686572650042696E61727920436C6F635F
:1017E0006B004469676974616C20436C6F636B00C4
:1017F000506C6179204D6F6465004C4544205469FC
:101800006D65005761726E696E6773004F6E20538D
:10181000637265656E204D656E75005468616E6B10
:1018200020596F750042692D48657820436C6F63BD
:101830006B00446179206F66207468652057656588
:101840006B0043616C6962726174696F6E205363EF
:101850007265656E005465726D696E616C005363EC
:101860006F72653A2020323333303000566563742E
:101870006F722047726170686963730048656C70AD
:101880002053637265656E004275726E496E20501A
:10189000726576656E74696F6E00416C736F20536C
:1018A0007570706F7274656400475053204E4D45DB
:1018B000412050617273696E67004461796C696799
:1018C000687420536176696E672054696D650041C4
:1018D0006C61726D00333720436F6D62696E6174A5
:1018E000696F6E7300546869732064656D6F206D55
:1018F0006F64652073686F777320736F6D65206FF9
:101900006620746865206361706162696C697469DE
:101910006573206F66207468650D0A415652204336
:101920006C6F636B2E205468652064656D6F20704A
:10193000726573657276657320746865207374616F
:101940007465206F6620796F757220636C6F636BAE
:101950000D0A00000000FF00FFFFFFFFFFFF00FF78
:101960000000005E6A695D695D6F676F675E6A6946
:101970005D80508050875B875B6F678050854887AC
:101980005B905A7C02830783078B028B0286098651
:10199000098B118B11830C830C7C117C11810981C3
:1019A000097C0284528B578B57935293528E598ED7
:1019B00059936193618B5C8B5C84618461895989E3
:1019C00059845272C079C579C581C081C07CC77CF9
:1019D000C781CF81CF79CA79CA72CF72CF77C777E3
:1019E000C772C016F419F619F61DF41DF41AF71A89
:1019F000F71DFB1DFB19F819F816FB16FB18F71855
:101A0000F716F4871E8E238E23961E961E9125911F
:101A100025962D962D8E288E28872D872D8C258C0A
:101A200025871E3E8A438D438D498A498A448F44C7
:101A30008F49954995439043903E953E95418F41FE
:101A40008F3E8AA2A8A9ADA9ADB1A8B1A8ACAFAC90
:101A5000AFB1B7B1B7A9B2A9B2A2B7A2B7A7AFA7A2
:101A6000AFA2A866DC6DE16DE175DC75DC70E3703A
:101A7000E375EB75EB6DE66DE666EB66EB6BE36BC2
:101A8000E366DC1A38213D213D29382938243F24DA
:101A90003F29472947214221421A471A471F3F1F22
:101AA0003F1A38A86EAF73AF73B76EB76EB275B228
:101AB00075B77DB77DAF78AF78A87DA87DAD75ADE2
:101AC00075A86E468647874A824B834E7E4F7F2D90
:101AD000D82ED94875497630D231D333CC34CD267F
:101AE000A627A76069616A41707000436C6F636BE1
:101AF0000043616C005465726D0047656E00426F73
:101B00006F740044656D6F00505053004E756D004A
:101B10004C6564004275726E696E004469616C00C8
:101B20004F6E004F66660031326872003234687260
:101B300000486578004461746500416C61726D0015
:101B40004469670042696E00526F6D004D696E0016
:101B50004D6F72736500446562756700506C617902
:101B6000004E6F726D005265760046460046520088
:101B70004E616D65004564697400446179004F00F1
:101B80005075736820533120746F205374617274E0
:101B900000475053004F6666002D3132002D313121
:101BA000002D3130002D3920002D3820002D372018
:101BB000002D3620002D3520002D3420002D33201F
:101BC000002D3220002D312000302020002B31202C
:101BD000002B3220002B3320002B3420002B35200B
:101BE000002B3620002B3720002B3820002B3920EB
:101BF000002B3130002B3131002B31320044535453
:101C0000004368726F6E6F005265736574003148EF
:101C10007A0034303936487A0042617564003139CF
:101C20003230302000323838303020003338343011
:101C30003020003537363030200031313532303009
:101C40000032353030303000343830302020003928
:101C500036303020200031343430302000555341AC
:101C60000045550035003600370038003900300097
:101C70003100320033003400271B2C1B481B401B53
:101C8000441B4C1B271B2C1B311B351B3A1B231BD6
:101C9000201B501B561B231B1E1C251C2C1C331CDD
:101CA0003A1C411C481C4F1C561C231B201B0E1C9D
:101CB000121CB91BBD1BC11BC51BCD1BD11BD51BCA
:101CC000D91B007FFCFDFEFF010203040203040593
:101CD000FF0607080900611B661B6A1B6D1B201BA2
:101CE000231B751B7A1B7E1B5D1C611C231BEB1ABF
:101CF000F11AF51AFA1A031BFE1A8234EC36690639
:101D00002634E1367106E632693679069033AA3612
:101D100081062033443289060333703691065833E6
:101D20008D3699060B34D636A106E933CB36A90693
:101D3000C733C036B106AD33B536B9063D3382364A
:101D4000C10673339836C906B9324A36CD06873292
:101D5000A6340000292A663601802A2B61320280CF
:101D60002B2C6A3203802CB1703200002D2EBC3136
:101D7000EA042E2F6132E2042F306A32DA0430B1E5
:101D8000703200003475BE31EA0435766132E20407
:101D900036776A32DA0437B17032000012136636D1
:101DA00005801311003204801195063200001510D1
:101DB0000C32018010941C3200001428D93100002C
:101DC000383966360180393AE23102803A3BEC31EB
:101DD00003803BBCF63100003C282E32000031323B
:101DE000D531F20432B35632000033002232000003
:101DF000DF0619EBF406A9EB0C1B03C3000033C389
:101E00001B1B86C30000C2C3911B03AA000033AA98
:101E1000FD1B86AA0000B6AAE71A039100003391C1
:101E2000081B86910000B691011C037800005778CA
:101E30003A1B86780000CE78101B035F0000335FEA
:101E4000141B865F0000DA5F5C1B034600003F4600
:101E5000081C86460000CE46191C032D0000392DB3
:101E6000701B862D0000C22D9C070314244750527E
:101E70004D432C0065D011241FBECFEFD8E0DEBF4C
:101E8000CDBF17E0A0E0B1E001C01D92AC3DB107AD
:101E9000E1F70E94CA2A0C94F73A0C9400001092C1
:101EA000B90081E18093B8000895982F84EA809367
:101EB000BC008091BC0087FFFCCF8091B900887F77
:101EC000883021F0803111F081E008959093BB00BB
:101ED00084E88093BC008091BC0087FFFCCF909188
:101EE000B900987F983111F480E0089580E0903433
:101EF00009F081E00895D9CF84E98093BC008091F6
:101F0000BC0084FDFCCF08958093BB0084E88093DF
:101F1000BC008091BC0087FFFCCF8091B90090E0AD
:101F2000887F883209F091E0892F089584E88093B2
:101F3000BC008091BC0087FFFCCF8091BB0008955E
:101F40002227E0E0F1E03DB74EB72193E317F40715
:101F5000E1F7089584B18F6084B987B18F6087B944
:101F60008AB188638AB95D9A5B9A579A5C9A5F983E
:101F70000895682F690D5B9865B9629568B95C989A
:101F80005C9A672F6A0D5B9A65B9629568B95C982F
:101F90005C9A5D985D9A0895672F690D5B9865B9A5
:101FA000629568B95C985C9A682F6A0D5B9A65B90E
:101FB000629568B95C985C9A5D985D9A0895809185
:101FC00054068823B9F098E09924AA2480916107E7
:101FD00070915C042091110530917C07D8D08091DC
:101FE000130570917E042091120730911E05CFD009
:101FF0009A9551F708959CE0A5E5B6E03FD092E0B0
:102000004AD0A0918C04B0918D041196A0938C04B9
:10201000B0938D040895EDE4F2E09924AA249AD0B7
:10202000A0918C04B0918D041196A0938C04B09370
:102030008D04089590915A04A2EDB4E0ED91FD91C4
:102040009D90970CAD90A80C0E2E0F2A09F082D00F
:102050009A95A1F7B4DFA2EFB4E095E00FD0A6E027
:10206000B5E092E018D0A0918C04B0918D04119647
:10207000A0938C04B0938D045F980895ED91FD9129
:102080009D90970CAD90A80C0E2E0F2A09F0C8D089
:102090009A95A1F70895ED91FD919D90970CAD90C3
:1020A000A80C0E2E0F2A09F0B2D09A95A1F7089528
:1020B000A5E5B6E09EE1E2DF91E0EDDFA0918C04C2
:1020C000B0918D041196A0938C04B0938D04089563
:1020D000A3E9B4E090911005DF93CF93C5EED6E06D
:1020E000ED91FD919D90970CAD90A80C099000206A
:1020F00009F48DD09A95A1F7CF91DF919091530675
:10210000992331F0A0917C04B0917D0491E0C3DF6C
:10211000809179049927972CA82CA0E0B1E0880F32
:10212000991F880F991FA80FB91F9091D004992368
:1021300039F08D917D912D913D9129D09A95C9F7D6
:10214000A0918C04B0918D041196A0938C04B0934F
:102150008D04089585918823E9F38B3071F0759192
:102160002591222309F4F6CF2F3F81F035913F933B
:102170002F930DD08F917F91F3CFA5908591292D2D
:1021800058D0922E85918F3F09F0E5CF0895AF0189
:10219000E9EBFFE0532E571A08F45194422E481AE7
:1021A00008F44194451440F4ECECFFE087277827CD
:1021B0008727232732272327281730F48227282729
:1021C0008227732737277327422E481A532E571A10
:1021D00008F45194222433246624731710F4639472
:1021E00001C06A94281780F05F9A0995250C311C6C
:1021F000022C020C041431041CF0760D2418310852
:10220000839511F0281788F75F98FA01089561E027
:1022100060937B048191882311F00BD0FBCF08954C
:1022200061E060937B048591882311F002D0FBCF9D
:1022300008952F0187FD59C0815208F456C0482FD8
:102240005527440F551F440F551F440F551FEEECE3
:10225000F4E1E40FF51F68E01F9360907B046620B3
:1022600021F149B14F77342F3F7D542F577E142FE2
:102270001F7EFF93EF936590772767FC4BD071E04B
:1022800066FC48D072E065FC45D073E064FC42D047
:1022900074E063FC3FD075E062FC3CD06A9559F76E
:1022A000EF91FF9168E010927B0449B14068342FB0
:1022B0003F7D542F577E142F1F7E6590662091F02E
:1022C000772767FC2BD071E066FC28D072E065FCB4
:1022D00025D073E064FC22D074E063FC1FD075E06D
:1022E00062FC1CD06A9549F71F915F98F201893111
:1022F00011F488E00DC0803811F484E009C08C30FE
:1023000011F48AE005C08B3011F486E001C08CE046
:10231000980E089503D07F917F91C2CF062E770F3C
:10232000790D372E3294660F6A0D262E229475B9D8
:1023300038B85BB94BB965B928B81BB94BB93BB9CB
:102340004BB97395372E329475B938B85BB94BB920
:1023500065B928B81BB94BB93BB94BB97A95372E3B
:1023600032946395262E229475B938B85BB94BB96F
:1023700065B928B81BB94BB93BB94BB97395372E22
:10238000329475B938B85BB94BB965B928B81BB97F
:102390004BB93BB94BB9602D0895282F3AE1839F83
:1023A0001A943AE0812D839F112420192A3010F0CD
:1023B0002A5083950895F1DF8A300CF081E08295F0
:1023C000822B08950E94902281E30E94F321FC0158
:1023D0006624552482E5282E87E2382E44245B9813
:1023E0005D985F9A1BB1012F0F7E520C631CE41D98
:1023F000008005B8029408B80BB91BB9F6CF622D5E
:10240000732D842D99270895262E372E482E089552
:102410008AE0280E311C411C089584E6280E311CE8
:10242000411C08959AE0F9DF9A95E9F787E0280EB4
:10243000311C411C089594E69F93F4DF9F919A9577
:10244000D9F7822D8951282E31084108822D8A50D2
:10245000282E310841080895822D8456282E3108EF
:10246000410808959AE0F8DF9A95E9F7822D8750A0
:10247000282E31084108089594E69F93F3DF9F9139
:102480009A95D9F785E2280E311C411C08955A9A75
:1024900080918B07882311F482E001C083E0809350
:1024A00069000895E89808951F920F920FB60F9251
:1024B00011248F939F9380915D048823F1F0809184
:1024C0008807882399F080912F039091300301971A
:1024D0009093300380932F03892B79F48091270305
:1024E000909128039093300380932F03F29A1092D7
:1024F00013078091100780937A049F918F910F901A
:102500000FBE0F901F90189514BC85E085BD8FE716
:1025100087BD0895F19A10920103109234038FEF52
:1025200080933603809303031092350310920203C5
:1025300082E085BB80936E00089510926E0008952E
:102540000F93FC018081882359F081508083882378
:1025500039F4002329F48EB3822B8EBB11821382AF
:1025600083B1862390E009F091E08281880F892B66
:102570008283803841F48181882399F581E08183C9
:102580008DE780832EC08F3789F48381882329F0DB
:1025900013828EB32095822305C08181882319F090
:1025A0008EB3842B8EBB118210821BC08823C9F48A
:1025B00085818823B1F08EB3822399F083818823AB
:1025C00031F491E091838FE0848393830AC0848106
:1025D00081508483882329F48EB3842B8EBB8FE0B3
:1025E00084830F9108951F920F920FB60F921124BA
:1025F0000F932F933F934F935F936F937F938F939B
:102600009F93AF93BF93EF93FF9316BC789481E0B1
:1026100093E060E148E020E100916D0791DF84E301
:1026200093E060E240E220E400E08ADF809136033C
:102630009091030389238F3F11F4F1987EDFFF917E
:10264000EF91BF91AF919F918F917F916F915F912A
:102650004F913F912F910F910F900FBE0F901F90B0
:10266000189510922A031092290310923B0410929D
:102670003A041092850010928400EFE6F0E0808129
:10268000826080830895EFE6F0E080818D7F808313
:10269000089584E08093810086E195E0909389001D
:1026A00080938800DECF3FB7F8942CE3829FC0016F
:1026B000112490932A03809329033FBF089580E15A
:1026C0009EE090933B0480933A041092D1060895C3
:1026D0001F920F920FB60F9211242F938F939F93F7
:1026E0002BB15F981092850010928400809129038D
:1026F00090912A03009729F0019790932A038093E1
:10270000290380913A0490913B04009751F001977E
:1027100090933B0480933A04892B19F481E08093D1
:10272000D10680917A04882361F0815080937A04E5
:10273000882339F481E08093F60680911007809316
:102740007A0480918304815080938304882321F448
:10275000F79A8FE08093830480916007882329F0A3
:102760008091600781508093600780915D04882389
:10277000E9F09091760480918004891790F480911B
:102780001805863048F0809113078C3328F481E0D7
:102790008093110710921805809118058F5F809320
:1027A0001805809113078F5F809313078BB12078F2
:1027B000282B2BB99F918F912F910F900FBE0F90C7
:1027C0001F9018951092B20082E087BB8093700032
:1027D0000895E0E7F0E080818D7F80830895109276
:1027E000B00087E08093B10081E68093B300089544
:1027F000569A5E98089580918407882309F44E9A2A
:1028000008955E9A08955E980895882309F0F9CF97
:10281000FACF84B18F7C84B985B1806385B908957E
:10282000F999FECF92BD81BDF89A80B50895F999C6
:10283000FECF92BD81BD60BD8FB7F894FA9AF99A28
:102840008FBF08959C0180916D07882311F4C90101
:10285000EECF0895A89584B7877F84BFE0E6F0E0C7
:1028600080818861808310820895F894809160004F
:102870008861809360008AE080936000FFCF4FB74B
:10288000F89490E0BC01660F771F680F791F9B01D9
:1028900028593F4FF901859194919093C5008093F9
:1028A000C40066597F4FFB018491882321F08091F9
:1028B000C000826003C08091C0008D7F8093C00003
:1028C0004FBF08951092C00098ED9093C10096E01C
:1028D0009093C200D4DF81E0809331030895109279
:1028E000C0001092C1001092C200109231030895EE
:1028F0001F920F920FB60F9211248F939F93EF9315
:10290000FF939091000380913303891721F481E0B4
:10291000809331030BC0E92FF0E0E95FFC4F808129
:102920008093C6009F5F9F7190930003FF91EF918A
:102930009F918F910F900FBE0F901F9018951F922F
:102940000F920FB60F9211242F933F938F939F9363
:10295000EF93FF933BB15F98909132039F5F20917B
:10296000C60080912C03891751F491E0909362077F
:1029700080918F078823A9F09093670712C0E09198
:102980003203F0E0E65CFC4F2083F09A2A3039F401
:1029900080918F07882319F081E0809367079093D7
:1029A000320380911A05882339F080916C078823BF
:1029B00019F482E08093700080912D0390912E0392
:1029C000019690932E0380932D038BB13078382B92
:1029D0003BB9FF91EF919F918F913F912F910F9074
:1029E0000FBE0F901F9018951F93182F80913103E1
:1029F000882399F4909133039F5F9F718091000326
:102A0000891781F46623B1F0E0917F07F091800788
:102A10000995809131038823B9F310923103109303
:102A2000C60008C0E0913303F0E0E95FFC4F10837B
:102A3000909333031F910895CF93DF93EC0102C06D
:102A400061E0D2DF89918823D9F7DF91CF91089592
:102A5000CF93DF93EC0103C061E0C6DF2196FE0156
:102A600084918823C9F7DF91CF910895F09BFECF21
:102A7000E0912C03F0E0E65CFC4FE08180912C03B8
:102A80008F5F80932C039091320380912C039817D1
:102A900009F4F0988E2F0895DC013FB7F894209147
:102AA000320390912C0380E0E92FF0E0E65CFC4FCC
:102AB000E0819F5F8F5F681708F0ED93EA3011F0B7
:102AC000291791F711971C92291709F4F098909300
:102AD0002C033FBF0895F09B17C03FB7F894209197
:102AE000320390912C03E92FF0E0E65CFC4F8081EB
:102AF0009F5F8A3019F02917B1F702C0291709F42E
:102B0000F09890932C033FBF0895109233031092D6
:102B10000003809131038823E1F308951F920F92FF
:102B20000FB60F9211242F933F934F935F936F93A0
:102B30007F938F939F93AF93BF93EF93FF931092E5
:102B4000B20080911A05882311F00E945822FF914B
:102B5000EF91BF91AF919F918F917F916F915F9115
:102B60004F913F912F910F900FBE0F901F9018958E
:102B70000FD7E89A0895E2E3F2E0E80FF11DE4913F
:102B80008E2F089508950895FC018581882319F4F6
:102B900083E6858302C08150858385810895FC0189
:102BA00080818F5F8C3308F080E080830895FC0182
:102BB00081818F5F8C3308F080E081830895FC0170
:102BC00082818F5F883108F080E082830895FC0164
:102BD000862F81508C3008F061E06483862F089541
:102BE000FC0164816F5F6483F2CFFC01643608F0FE
:102BF00060E06583862F0895FC0165816F5F6583C2
:102C0000F4CF8C3310F080E008958093840408950D
:102C10008C3310F080E00895809385040895883106
:102C200010F080E00895809386040895FC01262F1B
:102C3000643658F4862F6AE00E94FC39805D8193E7
:102C4000822F0E94FC39905D91938E2F9F2F0895C3
:102C50000F931F93CF93DF93EB016B81E7DFDC01D1
:102C60009DE29C93EC81E150F0E0EE0FFF1FEE0F30
:102C7000FF1FAF014D575F4FFA01849111968C935E
:102C800011979A012F5F3F4FF901849112968C930F
:102C90001297FA013296E4911396EC9313971496D7
:102CA0009C93149782E315968C93159780E3169660
:102CB0008C931697CD0107966D81B8DFDF91CF9188
:102CC0001F910F91089564E874E0C2CFFF920F93B3
:102CD0001F938B01FB016281A9DF0F2EFAE3FF2E08
:102CE000F02DFC01F192CF01F80161819FDFFC0121
:102CF000F192CF01F801608199DF1F910F91FF9050
:102D0000089564E874E0E2CFFF920F931F938C0163
:102D1000F62E862F82958F702EDFF80180838F2DFF
:102D20008F7029DFF80181830E5F1F4F802F912F55
:102D30001F910F91FF900895282F22952F709AE0F0
:102D4000299F900111248F70820F0895DC01149641
:102D5000EC911497E150F0E0EE0FFF1FEE0FFF1F14
:102D6000EA57FF4F84918C3151F415968C9190E085
:102D700083709070892B11F48DE108958CE1089592
:102D8000CF93DF93EC018B8181508B83882361F497
:102D90008C8181508C83882321F48CE08C83CE013C
:102DA000F3DECE01D3DF8B83DF91CF9108951F93A4
:102DB000162F662321F0CADF811708F410E0812F57
:102DC0001F9108951F93CF93DF93EC01162FEFDF30
:102DD000882309F411E01B83812FDF91CF911F918C
:102DE0000895FC0163816F5F6383ECCFCF93DF9322
:102DF000EC01F7DF813031F4CE01F2DE813011F4E5
:102E0000CE01FADEDF91CF910895E1EEF6E0808108
:102E10008F5F8083883120F01082CF010297E6CF48
:102E200008951F93DC0115962C911597822F6CE065
:102E30000E94FC39592F14963C911497832F90E0EF
:102E400087509F4FFC01149113964C91822F90E074
:102E500083709070892B29F4832F8150823008F47D
:102E60004150822F6CE00E94FC39252F30E0280F62
:102E7000311D2A5F3F4F852F86958695B901680FD2
:102E8000711DCB0167E070E00E941C3A90E0810F59
:102E9000911D67E070E00E941C3A90E0840F911D44
:102EA00067E070E00E941C3A1F910895EF92FF9234
:102EB0000F931F937C01862F90E009966CE070E0E1
:102EC0000E941C3AE82F6AE00E94FC39E81AF108D7
:102ED000042F10E0015010408DE691E09C01E29E2D
:102EE000C001E39E900DF29E900D1124080F191F52
:102EF000C7019695879596958795080F191FC70165
:102F000060E971E00E94083A060F171FF0E082E3C3
:102F100091E09C01E29FC001E39F900DF29F900D14
:102F2000112405966AE070E00E941C3A060F171FF4
:102F3000C70164E670E00E94083A061B170B20E008
:102F400030E0602F712F822F932F1F910F91FF90F0
:102F5000EF900895882399F080917604E82FF0E0AF
:102F6000E770F070EC5DFD4FE4918695869586954F
:102F7000A2EBB7E0A80FB11D8C91E82BEC938091E8
:102F800076048F5F8093760408950F931F93082F24
:102F9000882331F010E080E0DDDF1F5F1017D8F3E9
:102FA0001F910F91089581E0D5DF80E0D3CF81E0BC
:102FB000D1DF81E0CFDF81E0CDDF80E0CBCF0F93A9
:102FC0001F93CF93DF9395E0899FC00111248C015B
:102FD0000550194FC0E0D0E0F801EC0FFD1FE4915F
:102FE000EE2311F0E4DF01C0DEDF2196C530D1050C
:102FF00099F7DF91CF911F910F910895813831F4A6
:10300000D6DFD1DFD4DFCFDFD2DFCDCF823831F4CE
:10301000CEDFCDDFCCDFC7DFC6DFC5CF089510928E
:10302000760410928004109218058BE1E2EBF7E031
:10303000DF011D928A95E9F70895EF92FF920F93B1
:103040001F938091B1078F5F8093B107863109F09C
:1030500057C01092B10780918407813009F050C0A9
:103060000E945E23882309F04BC0D9DF81E8C6DFC8
:1030700086E08BDF0F2EF6E8EF2EF4E0FF2EF02D2A
:10308000F70180816AE00E94FC3999DF82E07DDFF0
:10309000F70180816AE00E94FC39892F90DF86E089
:1030A00074DF82E8ABDF86E070DFF70182918F0189
:1030B0006AE00E94FC3983DF82E067DFF8018081EB
:1030C0006AE00E94FC39892F7ADF86E05EDF82E8C1
:1030D00095DF86E05ADF8EEF9FEFE80EF91EF701CD
:1030E00080816AE00E94FC396ADF82E04EDFF701EE
:1030F00080816AE00E94FC39892F61DF86E045DF2C
:103100001F910F91FF90EF900895CF93DF93EC0103
:10311000442311F4FC0113C083E0683E780710F0EB
:10312000FE0103C0FE0180E381936436710510F453
:1031300080E381936A30710510F480E38193CB01C1
:10314000BF014AE050E00E94D33AEC2FFD2FDF018F
:103150000D900020E9F71197AE1BBF0B9E012A0FBF
:103160003B1F822F932FDF91CF910895BF92CF9273
:10317000DF92EF92FF920F931F93DF93CF93CDB720
:10318000DEB769970FB6F894DEBF0FBECDBFB82E7D
:10319000998F6B01C801A0E0B0E08D8B9E8BAF8B47
:1031A000B88FC901A0E0B0E0898B9A8BAB8BBC8B48
:1031B000CA01A0E0B0E08D879E87AF87B88BBC01C5
:1031C000CD0120EA35E140E050E00E94DD39EE24F7
:1031D000FF2487017601E60EF71E081F191F698973
:1031E0007A898B899C8920E83CE140E050E00E948C
:1031F000DD39E60EF71E081F191F6D897E898F893C
:10320000988D20E932E040E050E00E94DD39A801CD
:103210009701260F371F481F591F29873A874B8769
:103220005C8769897A898B899C8928E135E240E04D
:1032300050E00E94DD397B018C016D857E858F8594
:10324000988926E030E040E050E00E94DD39E60E4B
:10325000F71E081F191F6D897E898F89988D27EFAA
:103260003DE140E050E00E94DD39E60EF71E081F08
:10327000191F69857A858B859C8520E137E240E0BE
:1032800050E00E942F3AD801C701820F931FA41F5C
:10329000B51F8D839E83AF83B8876D897E898F89A3
:1032A000988D2DE832E140E050E00E94DD397B014D
:1032B0008C0169897A898B899C892AE230E040E017
:1032C00050E00E94DD39E60EF71E081F191F6D81C0
:1032D0007E818F81988520E137E240E050E00E94B6
:1032E0002F3AD801C701820F931FA41FB51F8983EE
:1032F0009A83AB83BC83BC01CD0120E137E240E07F
:1033000050E00E942F3A69017A016D897E898F8988
:10331000988D29E131E040E050E00E94DD39C60E91
:10332000D71EE81EF91E0B2D198D84E2D8018D934E
:103330008D01C701B60120E137E240E050E00E9474
:103340002F3A9B01AC01C801B90140E0DEDE8C01DF
:1033500069817A818B819C8120E137E240E050E0F5
:103360000E942F3A9B01AC01C801B90141E0CDDEBA
:103370008C016D817E818F81988520E137E240E06C
:1033800050E00E942F3A9B01AC01C801B90141E015
:10339000BCDE8C0169857A858B859C8520E137E2CE
:1033A00040E050E00E942F3A9B01AC01C801B901F6
:1033B00041E0ABDE69960FB6F894DEBF0FBECDBF1D
:1033C000CF91DF911F910F91FF90EF90DF90CF9001
:1033D000BF900895BF92CF92DF92EF92FF920F932A
:1033E0001F93DF93CF93CDB7DEB7EC970FB6F8946A
:1033F000DEBF0FBECDBF9E8F8D8F78A36F8FDC0198
:1034000015968C91159790E08053984F14966C9177
:10341000149713964C914ADD7B018C0187ED97E060
:103420006AE046E143DDE616F7060807190720F4CF
:10343000EF8DF8A11082F6C19701261B370BA90169
:1034400060E070E080E090E0A0E0B0E029A35AA343
:103450006BA37CA38DA39EA3AFA3B8A7352F462F44
:10346000572F682F792F8A2F9B2F0F2EFBEAAF2E15
:10347000F02D0F2EF0E3BF2EF02D0F2EF6E1CF2E04
:10348000F02D0F2EF5EFDF2EF02DEE24FF2400E0BF
:1034900010E00E94EA38F82F822F87588AABE1E0CB
:1034A000821708F0E0E0A32FA65EABAB21E0A317E4
:1034B00008F020E0BBA9EB0F31E0EB1708F030E09B
:1034C000232BEBABE42FEB52ECAB31E0E41708F02D
:1034D00030E04CA9420F21E08CA9481708F020E009
:1034E000322B4CABA52FA156ADAB21E0A51708F0B0
:1034F00020E04DA9430F31E0BDA94B1708F030E0A3
:10350000232B4DABE62FE55CEEAB31E0E61708F080
:1035100030E04EA9420F21E05EA9451708F020E0F7
:10352000322B4EAB672F685F6FAB21E0671708F057
:1035300020E04FA9430F31E07FA9471708F030E0A2
:10354000232B4FABF8AF81E0FF1708F080E038ADD8
:10355000320F21E0A8AD3A1708F020E0822B38AFF7
:10356000890F89AFED8DFE8D92818CE3989F90013C
:1035700011248181280F311DA90160E070E080E0F5
:1035800090E0A0E0B0E029A75AA76BA77CA78DA781
:103590009EA7AFA7B8AB352F462F572F682F792F8F
:1035A0008A2F9B2F0F2EFBE2AF2EF02D0F2EF2E96C
:1035B000BF2EF02D0F2EFBE2CF2EF02DDD24EE24BA
:1035C000FF2400E010E00E94EA38B92FAAA9A20F58
:1035D000E1E09AA9A91708F0E0E0FBA93F0F21E07C
:1035E0003F1708F020E0FE2FF30FE1E0F31708F09B
:1035F000E0E02E2B3F2F9CA9490FE1E0491708F08E
:10360000E0E0F22FF40F21E0F41708F020E0E22BC5
:103610004F2FFDA95F0F21E05F1708F020E0FE2F7C
:10362000F50FE1E0F51708F0E0E02E2B5F2F9EA9E3
:10363000690FE1E0691708F0E0E0F22FF60F21E0F2
:10364000F61708F020E0E22B6F2FFFA97F0F21E093
:103650007F1708F020E0FE2FF70FE1E0F71708F0E2
:10366000E0E02E2B7F2F98AD890F91E0E8AD8E170B
:1036700008F090E0E22FE80F21E0E81708F020E0E2
:10368000922B89AD8B0F1A2F032FF42EE52ED62EF9
:10369000C72EBE2E980F99ABAD8B3E8B4F8B588F9C
:1036A000698F7A8FEB8F9C8F80919A0790919B07FF
:1036B00090FF7AC0AD8DBE8D6C9170E080E090E09F
:1036C00027EE39EB40E050E00E94DD399B01AC0170
:1036D000550F220B322FA901322F2AAF2BAF2CAF5F
:1036E000512F560FF1E0511708F0F0E0B02FB70F4F
:1036F000E1E0B01708F0E0E0AF2FAB0FF1E0AB175F
:1037000008F0F0E0EF2BBA2F7F2D780FF1E07F1556
:1037100008F0F0E0AE2FA70FE1E0A71708F0E0E017
:10372000FE2B7A2F6E2D690F81E06E1508F080E078
:10373000F60FE1E0F61708F0E0E08E2B6F2F4D2D2D
:10374000430FE1E04D1508F0E0E0F82FF40F81E0C1
:10375000F41708F080E0E82B4F2F3AAD3C0D81E0E4
:103760003C1508F080E0FE2FF30FE1E0F31708F0BE
:10377000E0E08E2B3F2F2BAD2B0D91E02B1508F0A9
:1037800090E0E82FE20F81E0E21708F080E0982B4C
:1037900089A9FCAD8F0F890F5D8BBE8B7F8B688FE6
:1037A000498F3A8FEB8F8C8F6D897E894F89588D29
:1037B000298D3A8D0B8D1C8D7E010894E11CF11C26
:1037C000C701D4DCF70101900020E9F73197EE1929
:1037D000FF093E2F31502E2F2D5FEF8DF8A1E20F04
:1037E000F11D118240E087015CE2EF8DF8A1E20F4C
:1037F000F11DD801A30FB11D8C91808331503F3F43
:1038000089F021504F5F842F63E00E94FC39992397
:1038100061F7332351F3EF8DF8A1E20FF11D5083CF
:103820002150E3CFEC960FB6F894DEBF0FBECDBFAC
:10383000CF91DF911F910F91FF90EF90DF90CF908C
:10384000BF900895DF92EF92FF920F931F93CF9353
:10385000DF93C1E8D7E000E010E0DD240F2EFBE9A4
:10386000EF2EF7E0FF2EF02DC8010E9410148F3FBD
:1038700009F48D2D88830F5F1F4FCE15DF0511F0E2
:103880002196F2CFDF91CF911F910F91FF90EF9092
:10389000DF900895EF92FF920F931F93CF93DF93E2
:1038A00001E817E0C0E0D0E00F2EFCE9EF2EF7E0D2
:1038B000FF2EF02DCE016FEF0E942214F80111921D
:1038C0008F012196EE15FF05A9F7DF91CF911F918A
:1038D0000F91FF90EF9008950C944F0FEF92FF928D
:1038E0000F931F93F82EE62E1FEF80ED0E94550FC9
:1038F000882319F00E947C0F14C08F2D0E94840F22
:10390000882319F00E947C0F0CC08E2D0E94840F1A
:10391000082F882319F00E947C0F03C00E947C0F9F
:1039200003C0115011F706C0802F1F910F91FF9017
:10393000EF90089581E0809366070FEFF5CF8091B7
:103940006D078823D9F4809184048C3328F40E9475
:10395000DB11682F80E0C2DF809185048C3328F46E
:103960000E94DB11682F81E0B9DF809186048831E5
:1039700028F40E94DB11682F82E0B0CF0895809177
:103980008807882311F061E901C060E987E0A6CFCC
:10399000F6CF0F931F93082F1FEF80ED0E94550F56
:1039A000882319F00E947C0F16C0802F0E94840F7C
:1039B000882319F00E947C0F0EC081ED0E947B0FBE
:1039C000882319F00E947C0F06C00E94960F182FC2
:1039D0000E947C0F03C0115001F704C0812F1F917A
:1039E0000F91089581E0809366071FEFF7CF84E081
:1039F000D0DF8F73A1D9803208F081E080938704F3
:103A000085E0C7DF8F7198D9982F81508C3008F0EE
:103A100091E09093880486E0BCDF8ED9843608F06C
:103A200080E0E9E8F4E080833597CF016381BFD976
:103A3000882319F481E08093870408951F9380916F
:103A40006D07882309F5E7E8F4E01081CF010397BB
:103A5000612FADD9882339F0812F0E94DB11682FA7
:103A600084E03CDF01C0C3DF809188048D3028F4FE
:103A70000E94DB11682F85E031DF809189040E946C
:103A8000DB11682F86E02ADF1F9108950F931F93A3
:103A900006E814E0F80110821092850402501040EC
:103AA000F80110824CDF81E0F80184838383158262
:103AB000C5DF85E090E061E00E9422141F910F9124
:103AC0000895E6E8F4E08081815080838F3F31F4EF
:103AD00087E18083CF01029753D9B0DF30CFE6E88A
:103AE000F4E080818F5F8083873128F01082CF01DE
:103AF00002977CD9A3DF23CF1F93182F1F7780E075
:103B0000612FECDE82E045DF682F6F7B82E0E6DE2E
:103B1000812F1F9108950F931F93182F80E039DF95
:103B2000082F112319F088230CF4E6DF802F8F77FC
:103B300003D98C3308F080E0809384041F910F91A7
:103B40000895E9DF81E025DF8F77F6D88C3308F020
:103B500080E08093850482E01CDF8F73EDD888318C
:103B600008F080E0809386040895FC0180918C0722
:103B7000823021F085818850873008F08FEF0895DA
:103B80001092190510925E041092180710925904B1
:103B9000ECDFE82F8F3F61F180918C07882399F447
:103BA00082E0809319058BE080935904F0E0EA5F8E
:103BB000FE4FE4918E2F82958F7080935E04EF709C
:103BC000E09318070895813099F4809319058AE0ED
:103BD00080935904F0E0E25FFE4FE4918E2F8295CE
:103BE0008F70875E80935E04EF70E75EE093180746
:103BF00008951F93162FB9DF982F8F3F11F480E09F
:103C00000DC0113019F480918D0705C080918E0789
:103C100002C0915086959923E1F781701F91089514
:103C2000CF93DF93EC01A1DF8F3F59F18C8183307B
:103C300040F1833071F49B8180915E04981708F104
:103C4000981709F520E09A81809119059817E0F0FE
:103C50001AC0909159048917B0F0891791F49B818B
:103C600080911807981778F0981759F48A81823054
:103C700040F410925B04882331F081E080935B0470
:103C800002C020E001C021E0822FDF91CF91089592
:103C9000CF93DF93EC0169DF8F3F99F09091590446
:103CA0008C81981780F0981761F4909118078B8198
:103CB000981748F0981729F420E08A81823020F084
:103CC00002C020E001C021E0822FDF91CF91089552
:103CD0001F93162F4ADF8F3F11F480E01BC0E82F9F
:103CE000F0E0EC5DFD4F8491113041F460918D075F
:103CF000682B60938D078CE090E007C060918E0781
:103D0000682B60938E078DE090E00E9422140E9441
:103D10005B2E81E01F9108958FED96E031DF8FEDEE
:103D200096E07EDF882391F080915B04882311F474
:103D300081E008958FED96E062E05BDF882331F447
:103D40008FED96E062E0C4DF80E0089580E00895A2
:103D50001F93182F84E894E013DF84E894E060DF79
:103D6000813079F484E894E061E043DF882309F549
:103D7000112309F0B4DE84E894E061E0A9DF11E0EA
:103D8000E9CF84E894E084DF882399F084E894E024
:103D900061E02FDF882369F084E894E062E029DFA6
:103DA000813039F0112329F08CDE84E894E062E060
:103DB0008FDF1F91089581E0CBCF80E0C9CF1092B3
:103DC000CE0410929004809116078C7F8093160782
:103DD0000895DC01FC0180E061936F5F67FD60E2A4
:103DE0008F5F8431C9F754961C92862F0895E3E9BA
:103DF000F4E0AFE1B5E08DEE27E09FEFB183A08363
:103E000022838383825155969C9355973496569678
:103E1000813FA1F70895FC01DC0180E090E29D93D1
:103E20008F5F8431E1F7148A9F012A5E3F4FC901F9
:103E300008950F931F93CF93DF9360919304709134
:103E4000940480911005282F30E02150304040E04C
:103E500014C01196CD56DB4FFD01EE0FFF1FEE0F84
:103E6000FF1FED56FB4F8081918199838883AB5171
:103E7000B94F8C91F80180834F5FA42FB0E0ED0122
:103E8000CC0FDD1FCC0FDD1F8D010B51194FA21779
:103E9000B307FCF2CD56DB4F79836883CB01BBDFE0
:103EA00081E0F8018083DF91CF911F910F910895F8
:103EB0000F931F932FE135E010E001E009C0C90125
:103EC000AADF9C01E12FF0E0EB51F94F00831F5F67
:103ED00080911005181798F372DF1F910F910895C4
:103EE000E82F80911005E81708F0E0E0F0E0EE0F11
:103EF000FF1FEE0FFF1FED56FB4F8081918108954C
:103F00009091CE049F5F9093CE04809110059817F6
:103F100038F08FDF8091100581508093CE040AC065
:103F2000892FDEDF78DFE091CE04F0E0EB51F94F2E
:103F300081E0808310929004809116078C7F80939B
:103F4000160708951F93182F8091160780FF01C050
:103F5000D7DF8091160781FF05C08D7F80931607FC
:103F6000109290048091CE04BBDF20919004FC015C
:103F7000E20FF11D1083103231F0E091CE04F0E039
:103F8000EB51F94F1082809190048F5F80939004E1
:103F9000843128F0809116078160809316071F9165
:103FA0000895813F69F4862F90E0840F911D813838
:103FB00091050CF040E0609379044093D00408959B
:103FC000823F91F4643118F46093900402C010921F
:103FD000900480911005481710F44093CE0480910E
:103FE00016078C7F809316070895CF93DF93EB011C
:103FF000E881E7FD17C0F0E0EE0FFF1FEE0FFF1F97
:10400000DF01A050BF4F89818C938A8180951196E2
:104010008C931197EE5FFE4F8B8180838C8180950E
:1040200013968C93DF91CF910895833F61F490E0D4
:10403000611191E0990F990F809116078B7F892B61
:10404000809316070895843F09F5809116078860CC
:10405000962F91709295907F8F7E892B8093160773
:10406000662331F4109253068EE080931005089574
:1040700081E0809353068DE0809310058091CE04FB
:104080008D30E0F08CE08093CE040895853F89F474
:10409000809116078062962F91709295990F990FD3
:1040A000907C8F7B892B80931607662309F438C395
:1040B00027C3863F19F4662309F4FACE089581E9EF
:1040C00094E00C94DD381F938091910490919204B8
:1040D000892B99F51091CE04812F02DFDC01E3E4F6
:1040E000F4E08D9181938823E1F7E0919004E4312D
:1040F00010F0E3E106C08091160780FF02C0E111D5
:10410000E150F0E0ED5BFB4F8FE58083812F90E085
:10411000880F991F880F991F8D569B4F6FEF43E4AF
:1041200054E00E944C389093920480939104E09163
:10413000CE04F0E0EB51F94F10821F9108950F93D8
:104140001F930FE115E0C8016FED76E00E949C3AE5
:10415000F80101900020E9F73197E01BF10BCF0146
:10416000800F911F66E171E00E949C3A1092E50673
:1041700081E08093CE0461E308E016E10DC0019F69
:10418000C0011124815E9A4F24DE682FE02FF0E0F9
:10419000EB51F94F10820F5F80911005081778F3EB
:1041A0001F910F9108950BDE109279041092D004A4
:1041B00010924104809116078460877880931607D7
:1041C00080919A0784FF02C08EE001C08DE0809349
:1041D00010050DDE6DDEB3CF1F930E943615182F2C
:1041E00080914104813051F4173FE8F410932B0380
:1041F00082E0809341041092420474C0823069F5D9
:1042000080914204E82FF0E0E45CFB4F10838F5F65
:1042100080934204813051F480912B03833F08F452
:1042200061C0612F02DF109241045CC0823051F402
:1042300080912B03813F08F455C060913C04412FCD
:10424000B0DEF1CF853009F04DC080912B03803F67
:1042500051F76CE374E0C9DEE6CF1F3F31F481E033
:104260008093410410922B033DC01032B8F51830F2
:1042700041F4809190048823A9F1815080939004A7
:1042800031C01D30A1F48091160781FF01C038DED6
:104290009091160790FF07C080919004843110F12F
:1042A0009E7F909316078091160782600FC0193089
:1042B00011F480E216C01A3061F48091160780FF75
:1042C00001C01EDE8091160781608D7F80931607E6
:1042D00009C08EE537DE812F8F5B03C017FD02C05A
:1042E000812F30DE1F9108958091160783FF09C04A
:1042F00084FF0BC081E0809353068DE0809310050E
:1043000015C080919A0784FF04C0109253068EE076
:10431000F5CF81E0809353068DE080931005809166
:10432000CE048D3018F08CE08093CE0480919A07F3
:1043300085FF10C086E095E090937D0480937C0417
:1043400080910605909107059AD1809308051092F7
:10435000090508C08AE095E090937D0480937C0471
:1043600010920D058091160785FF03C086FD06C0DB
:10437000D7C180919A0786FD01C0D2C108950F93DD
:104380001F9388E690E19093800780937F07ACDFCE
:1043900082E48093600702E405D7F59B03C08FDEBB
:1043A0000E94F629F39B07C0F39889DEA9D1CDD5E9
:1043B0001F910F910895F09B0AC081DE1FEA0CDF68
:1043C000F09B02C01150D9F700936007E5CF8091B0
:1043D0006007882309F78091160782FF01C073DE0A
:1043E00010924104D9CF9EEF20E231E040E0A0E0FE
:1043F000B1E0813329F4F9012F5F3F4F949114C04C
:10440000823311F4942F10C0833349F447FD02C066
:104410009E5F0AC0403809F491E0925005C0843391
:1044200019F4942F990F990B9C934F5F51E0AF3F74
:10443000B50711F01196DDCF80E091E008950C945E
:1044400035140F931F930E9436150E943615082FBE
:104450000E943615182F0E943615682F712F802F55
:1044600090E00E9404121F910F910895FF920F9304
:104470001F930E94FF11F62E072F182F80E593EC53
:104480000197F1F786E40E94202C80E00E94202C06
:10449000812F0E94202C802F0E94202C8F2D0E9483
:1044A000202C8AE00E94202C1F910F91FF900895EC
:1044B0000E94E91381E080936C0778941D9902C0F3
:1044C0000E9435140E9436158D3219F40E9408128C
:1044D0001EC0843619F40E94121219C0843419F4D3
:1044E0000E941B1214C08B3219F40E9426120FC0B6
:1044F000853719F40E9432120AC0853519F40E94DA
:104500003C1205C0833711F49CDF01C06CDFAEDFC5
:10451000809131038823E1F3F89410926C07089599
:104520000E94192CF8940E9452120E949D120E941F
:1045300043130E94E91384E00E943F1481E08093BA
:104540001A057894089581E00895982F8091C0000D
:1045500085FFFCCF9093C6000895CF93DF93EC01C5
:1045600001C0F3DFFE01219684918823D1F7DF910A
:10457000CF910895CF93DF93EC0101C0E6DF8991DD
:104580008823E1F7DF91CF91089581E008958FEFBF
:1045900080930303809336038093650788E28093BA
:1045A00019078FE48093D10488E080935A048DE248
:1045B00097E09093D3048093D2041092120581E087
:1045C000809364078EE38093100780937A048FE0D2
:1045D0008093830484E18093B10708951092D804F6
:1045E00080918A07843019F420E030E01FC08330C6
:1045F00031F483E58093D8042AEA34E117C080912E
:104600008907853011F0833069F420910E053091CF
:104610000F05809186048C3048F020917D07309101
:104620007E0704C020910E0530910F053093D7040A
:104630002093D604089580918907863010F0109257
:10464000890780918907089580918A07863010F044
:1046500010928A0780918A0708958A3311F488E0BE
:104660000895803811F484E008958D3211F48AE0C1
:1046700008958C3211F08CE0089586E008950F9330
:104680001F93CF93DF938C01C0E0D0E003C0E5DF40
:10469000C80FD11DF80181918F018823C1F7CF3F49
:1046A000D10509F030F48FEF90E08C1B91099595BE
:1046B0008795DF91CF911F910F91089580911205F9
:1046C000811181E0089510927A0408958091100775
:1046D00080937A04089580916E07882381F48091F5
:1046E000CF048F5F87708093CF04E82FF0E0EE0F48
:1046F000FF1FE958FC4F85919491782E892E0895DB
:1047000080918707853059F010926E0790E00596EA
:104710006AE070E00E941C3A80937F04DCCF089529
:1047200081E080936E077724882410927F04089597
:1047300080918707853009F4F3CFE2CF809127037A
:10474000909128039093300380932F030895209134
:104750008807222349F02F3739F0822F90E027FD78
:104760009F6F8050904F02C080E090E190932803AB
:104770008093270308958EE097E00C94DD3885E55B
:1047800096E06DE274E048E350E00C94883AF894C7
:1047900080938807F4D8DBDFD1DF98DF7894089521
:1047A000682F8EEF94E04EE252E00C944C388091EA
:1047B000120581FD0CC080910E0790910F07892B87
:1047C00031F48FEFEDDF90930F0780930E0708957C
:1047D000682F8AEF94E04CE252E00C944C388091C0
:1047E00065078F3F79F481E08093650780911B0511
:1047F00090911C05892B31F480EFEADF90931C0522
:1048000080931B0508951F93182F809395070E948E
:104810008515812F0E943F141F9108951F93809149
:10482000F306282F30E040E050E080916D078823A8
:1048300011F041E050E0242B352B232B11F5809112
:104840009207882341F480E280939C0710929D0791
:1048500081E08093920781E190E0609192070E944D
:10486000221410E00AC0E12FF0E0CF014E96E4568A
:10487000F84F60810E9422141F5F809192071817E1
:1048800090F31F9108951F93682F192F80939A0713
:1048900090939B0789E190E00E9422148AE190E0C6
:1048A000612F0E94221481E01F910895682F809348
:1048B000870786E090E00E9422143ADF81E00895A5
:1048C000682F8093850784E090E00E94221481E0A5
:1048D0000895682F8093820781E090E00E9422145F
:1048E00081E00895FF920F931F938091920781506A
:1048F000843110F4FF2418C088E0809392078CE97B
:1049000097E06BEE76E00E949C3A81E08093F3069C
:1049100013C00F2D10E0C8014E960E9410140456CB
:10492000184FF8018083F394E0919207FE1688F304
:10493000F0E0E456F84F10821F910F91FF90089518
:10494000FF920F931F93F82E80919107813029F4E5
:10495000109207051092060533C0882339F48CE9BC
:1049600097E0909307058093060521C0833091F46A
:1049700084E894E00E941117E82FF0E0EE0FFF1F8B
:10498000E451FF4F6591749108EF16E0C8010E9451
:104990009C3A09C0843059F408EF16E084E894E0AA
:1049A000B8010E94EA19109307050093060580914B
:1049B00006059091070563DE80930805F0920905CE
:1049C0001F910F91FF90089584EA8093DC0482EC9C
:1049D0008093E0048EE58093E4048CE78093E80400
:1049E00087E18093EC0485E38093F00485EAA8DFF7
:1049F00089E598E09093D3048093D204EFDD809111
:104A00009A0790919B07969587959695879580959F
:104A1000817080935406089588EB8093DC048FECBA
:104A20008093E0048EE68093E40485E88093E804B4
:104A300080E28093EC0487E38093F00489E180DFD7
:104A400082E492E09093D3048093D204C7DD109265
:104A500054060895EAEDF4E0118210821282349631
:104A600084E0E23FF807C1F781E96ADF8DE297E071
:104A70009093D3048093D204B1DD1092540608952C
:104A8000682F80938B078AE090E00E9422140E9496
:104A9000351481E00895682F80938C078BE090E0B7
:104AA0000E94221488C91F93182F8093840788239B
:104AB00011F00E9403140E940F1884E18093B10743
:104AC00083E090E0612F0E94221481E01F910895FD
:104AD0009C0180918907823019F4C9010C948416D5
:104AE000C9010C941616809189078150823000F517
:104AF000809113078695982F969596956091130748
:104B0000680F690F96959695690F643608F064569C
:104B10008091120580FF03C083E6861B682F809179
:104B2000F4069091F506009719F0D2DFFC0110828F
:104B300008950F931F93CF93DF931091890715303A
:104B400019F4CFE6D7E05DC0133031F48FE697E07B
:104B50000E946316EC0155C01430D9F48FE697E03B
:104B600060919907B5DF1AE3FC011193CF016091C1
:104B70009807AEDFFC011193CF0160919707A8DF82
:104B8000FC0180E8808381E481838CE48283EF01EF
:104B900037C060918604112329F4E62FF0E0E15A32
:104BA000FC4F64918FE697E093DF0AE3FC010193E9
:104BB000CF01609185048CDFFC010193CF016091EE
:104BC000840486DFEC01112369F480E888838091F6
:104BD00086048C3010F080E501C081E489838DE487
:104BE0008A830EC080919407882359F011501230A7
:104BF00040F4FE010193F093F506E093F40673DFB1
:104C0000239618828FE697E090930B0580930A0510
:104C100036DD80930C05DF91CF911F910F910895A0
:104C2000682F8093940783E190E00E94221481DF33
:104C300081E0089580938907FEDC682F88E090E08A
:104C40000E942214CBDC75CF8093CB0472DF80915D
:104C5000CB04882361F1A2EDB6E0EFE6F7E08DE04A
:104C600001900D928150E1F78091CB04823019F4CC
:104C7000E5EDF6E019C0833019F4E8EDF6E014C074
:104C8000853041F480E28093D9068093DA06EBED1B
:104C9000F6E00AC0843019F0E2EDF6E005C080E2EB
:104CA0008093D506E6EDF6E080E280838183089567
:104CB000DF92EF92FF920F931F93CF93DF93082F12
:104CC000862F0E94DB11D82EC02FD0E082958F70E6
:104CD000E82FF0E0EE0FFF1F06E914E1E00FF11FEF
:104CE00025913491B2EDEB2EB4E0FB2EFE01EE0FD8
:104CF000FF1FEE0FFF1FEE0DFF1D20833183CF013D
:104D0000B9010E948934ED2DF0E0EF70F070EE0FE4
:104D1000FF1FE00FF11F25913491FE013196EE0F38
:104D2000FF1FEE0FFF1FEE0DFF1D20833183CF010C
:104D3000B9010E948934DF91CF911F910F91FF90AB
:104D4000EF90DF900895CF92DF92EF92FF920F9352
:104D50001F93CF93DF93E82E862F8A0169010E946B
:104D6000DB11F82ECE2DD0E082958F70E82FF0E089
:104D7000EE0FFF1FE00FF11F2591349102ED14E0BB
:104D8000FE01EE0FFF1FEE0FFF1FE00FF11F20834C
:104D90003183CF01B9010E948934EF2DF0E0EF702B
:104DA000F070EE0FFF1FEC0DFD1D25913491FE01FB
:104DB0003196EE0FFF1FEE0FFF1FE00FF11F208354
:104DC0003183CF01B9010E948934DF91CF911F91C6
:104DD0000F91FF90EF90DF90CF90089580918A0718
:104DE000833089F480919A0783FF09C0E09186049B
:104DF000F0E0E15AFC4FE49186E06E2F03C086E0BC
:104E00006091860455CF843041F486E06091860439
:104E10004BE752E02BE433E096CF809186046CE0C0
:104E20000E94FC3985E0989F9001112480918504AF
:104E30000E94FC39280F311DB901E3E0660F771F8E
:104E4000EA95E1F7620F731F67567E4E7093EB048D
:104E50006093EA048AEE94E00C94893480918A0786
:104E6000833021F484E06091850422CF843039F4CA
:104E7000609185044DEB52E02BE433E064CF609108
:104E8000850489E0689FB00111246358704F7093C6
:104E9000E3046093E20482EE94E00C948934809100
:104EA0008A07833009F02CC082E06091840400DF1F
:104EB000E091840489E0E89FF0011124E75AF74F5C
:104EC0008491809361073196849180935C0431963C
:104ED0008491809311053196849180937C0731965B
:104EE0008491809313053196849180937E0431964A
:104EF0008491809312073196E491E0931E05089502
:104F0000843041F482E0609184044DEB52E02BE464
:104F100033E019CF6091840485E0689FB0011124CB
:104F20006F5A714F7093DB046093DA048AED94E05A
:104F30000C948934B4DF92DF51CF109263074EDBBB
:104F4000F9DFF7DD80910905FBCC1F937DDB182F7E
:104F5000843091F489E78093F80491E09093F90408
:104F60008BE68093FC049093FD0487E88093000512
:104F70009093010551DD44C0833091F489E780931B
:104F8000F8049EEB9093F9048BE68093FC049093D5
:104F9000FD0487E8809300059093010515DD30C07E
:104FA000882319F485E79AE012C0813049F485E737
:104FB0009AE090930F0580930E0583E69BE00BC06B
:104FC000823019F487EC9CE002C08DEE9DE0909356
:104FD0000F0580930E0590937E0780937D0789E7E8
:104FE0008093F80494EB9093F9048BE68093FC048F
:104FF0009093FD0487E880930005909301052ADDD6
:105000009CDF812F1F910895682F80939107843032
:1050100021F480919A0781FF04C080E190E00E9412
:10502000221493CF80938A0790DF682F89E090E065
:105030000E942214D3DA7ECF41DB882329F40E9418
:10504000A11D0E94F71C79CF08951F93182F8091FE
:105050001205812781FF09C011FD02C08EE301C046
:1050600082E080937A04809310070E940F1884E1F5
:105070008093B10710931205DFDF1F91089580918F
:10508000120581FF05C08EE380937A048093100798
:1050900010921205D1CF0E94FB130E941D1880911F
:1050A00084048150809384048F3F59F0809163077A
:1050B000813009F442CFF3DE8091190784FD1DC0D1
:1050C00038CD2BE32093840491E090936A0780917C
:1050D00085048150809385048F3F71F4209385046B
:1050E00090936B07809186048150809386048F3F54
:1050F00019F487E18093860420CF08950E94FB1362
:105100000E941D18809184048F5F809384048C33E7
:1051100080F4809163078823C1F580919A0790916C
:105120009B0790FD32C0BBDE8091190784FD39C01A
:1051300000CD91E090936A071092840480918504D9
:105140008F5F809385048C33E0F090936B0710920F
:105150008504809186048F5F80938604883188F06F
:10516000109286048091190784FD04C084E894E0BD
:105170000E94F6168091120581FF07C00E94DB1E77
:1051800004C08091120581FF01C0D7CE0E949F1CF0
:105190008091190784FD04C00E94F71C0E94DB1E49
:1051A000CCCE089580919407882329F080918C04B7
:1051B000877009F498DCE0917F07F09180070995EA
:1051C000F19906C083B18073803311F00E948A1276
:1051D000F69B03C0F6980E9435148091110788232E
:1051E000E1F020918004822F90E0877090708C5DB8
:1051F0009D4FFC019491269526952695E22FF0E08F
:10520000EE54F84F808189230E9405148091800418
:105210008F5F8093800410921107F29B6AC0809187
:10522000140590911505A0911605B09117050196EA
:10523000A11DB11D8093140590931505A09316052B
:10524000B09317058091120580FF02C024DF01C0D2
:1052500055DF80916D0780FF09C081FD01C08BDAA9
:1052600080916D0782FF03C036DA01C084DA809135
:105270007504882389F59091860480919907981781
:1052800059F59091850480919807981729F5909188
:105290008404809197079817F9F4809185078823F3
:1052A000D9F480916D078823B9F480918A04909194
:1052B0008B04892B89F480911907883368F482ED77
:1052C00094E060EF40E050E00E944C3890938B04F3
:1052D00080938A040E945F1380918C0490918D04C6
:1052E000909378048093770410928D0410928C042C
:1052F000F2988091F606882361F01092130757DA2E
:105300008091120580FF02C0C6DE01C0F7DE109258
:10531000F606F79B03C00E94A838F79880912903EE
:1053200090912A03892B19F481E08093640780917E
:105330006A07882309F43EC080917F0481508093DE
:105340007F04882359F4C7D98091870790E0059698
:105350006AE070E00E941C3A80937F04809182078B
:10536000882309F0D9D410926A0780916B078823AB
:1053700009F120E030E080918407833011F421E0CE
:1053800030E08091820790E02823392380918507BF
:1053900090E028233923232B59F080918604843010
:1053A00039F482E095E060EF40E252E00E944C3830
:1053B00010926B078091D106882361F080918A0456
:1053C00090918B04892B31F010928B0410928A04F7
:1053D0001092D10680916207882339F0809184076A
:1053E000823009F44E9A109262070895EF92FF926C
:1053F0000F931F93DF93CF93CDB7DEB764970FB6AC
:10540000F894DEBF0FBECDBFF59880918A049091CD
:105410008B04892B29F08AE894E00E94DD386BC068
:10542000E0907F07F0908007AAD98091770490914F
:1054300078048E010F5F1F4FB8014AE050E00E94D0
:10544000D33AF80101900020E9F73197E01BF0E032
:10545000D801AE0FBF1F88E48C93DE01AE0FBF1FD3
:105460008AE712968C931297FD0113821093860699
:1054700000938506609114057091150580911605BD
:10548000909117058E01075F1F4FA8012AE030E0B9
:105490000E94B03AF80101900020E9F73197E01B33
:1054A000F0E0D801AE0FBF1F83E58C93EC0FFD1F1A
:1054B000128610938A06009389068BEF9FE09093E3
:1054C000800780937F0784E00E9453136BDE0E9465
:1054D00026378091290390912A03892B21F0F39993
:1054E00002C0F59BF3CFF59880E00E945313F09231
:1054F0008007E0927F0764960FB6F894DEBF0FBE78
:10550000CDBFCF91DF911F910F91FF90EF90089544
:105510008BE090E19093800780937F0743DEF59BBB
:1055200001C064DFF39B03C0F39880E0089580918D
:105530008F07882319F00E943D38F0CFF09BEECF03
:1055400075D4882359F381E008958AE190E190931E
:10555000800780937F0789E480930D0523DEF59B08
:1055600001C044DFF39B03C0F39880E00895F49BEF
:1055700003C0F4980E94553580918F07882319F055
:105580000E943D38EBCFF09BE9CF50D4882331F314
:1055900081E008951F93CF93DF930E942A1481E046
:1055A000809364001EBA882477240E94C7220E9438
:1055B0006C1C0E9484120E9449130E94EF130E94E7
:1055C000AA0F0E94F8130E9403140E9409140E945B
:1055D00088380E94221C2FD837D80E944712B7D88B
:1055E000ADD8A6D87FD980919507893038F0109230
:1055F000950784E190E060E00E9422148091950775
:105600000E94621480919607843030F085E190E02A
:1056100060E00E94221480E0809375040E94D320F1
:105620000E940F18ACD88BEF9FE090938007809377
:105630007F070E94C31580916607882331F480910B
:105640008607882311F40E94461D81E00E94A11D57
:105650000E94F71C80916607882371F410918404DE
:10566000A1DD81E00E948B1D809184041817C1F395
:1056700081508093840442DD0E94B81581E08093BC
:105680005D0478940E94DB1E60DCCDD381E0C8E528
:10569000D0E103C081E001C080E0D0938007C093D7
:1056A0007F070E940D3649DC80917504882311F430
:1056B0004CDF03C0813021F42BDF882359F7ECCF76
:1056C000823019F40E94BF21E7CF833019F40E9481
:1056D000E211E2CF843011F4A5D4DECF8530E1F6BB
:1056E0000E943514D9CF90E0880F991FFC01E6592C
:1056F000FB4F259134918E589B4FFC01A591B4919D
:105700008C9191E08927F9010995089590E0880F1F
:10571000991F82569B4FFC0125913491F9010995FF
:105720000895FC0180E28193CF010895982F81565E
:105730008A3108F49052892F0895CF93DF93EC01BA
:105740008881982F90539A3040F0603149F4EEDF11
:10575000982F8154863020F49753988381E001C0BC
:1057600080E0DF91CF91089584E295E00E942815B2
:1057700081E0089587E395E00C942815FBDF8FED19
:1057800096E00E94281582EB94E00E94281584EF91
:1057900096E00C942815F2DF87E595E00E94281525
:1057A00081E008950F931F93182F092F67E375E089
:1057B0000E949C3AA12FB02FFD0101900020E9F733
:1057C0003197EA1BFB0BE80FF91FCF011F910F91D7
:1057D00008950E944A1C0E94351481E0089580912A
:1057E0008207882331F080E00E94A11D0E94F71CEF
:1057F000A4DBC4DF81E008951F93CF93DF93EC0116
:1058000080918404182F125E1C3348F01C5307C08B
:10581000C9DC80918404811711F480E006C0F09BFC
:10582000F7CF0E943615888381E0DF91CF911F91D9
:10583000089501C0B7DC809131038823D9F308951E
:1058400061E00C94F414CF92DF92EF92FF920F93E9
:105850001F93DF93CF930F92CDB7DEB78EE195E024
:105860000E9428150CE917E0FF24EE246E0108942D
:10587000C11CD11CC601C0DF882321F40E94FC3466
:1058800080E03AC08981DCDF9F2D9F5F89818D3068
:1058900089F08A3079F0F80181938F01803211F01C
:1058A000EE2404C0EE2041F4EE24E394943121F080
:1058B000F92EE0CF2F2D01C0292F8D3049F08A30ED
:1058C00019F406C091508F01F80182918032D1F312
:1058D000222349F480919107882311F481E001C0CB
:1058E00080E092DB08C0F80110829093920710923A
:1058F000F3060E94A23481E00F90CF91DF911F91B7
:105900000F91FF90EF90DF90CF900895DF92EF928C
:10591000FF920F931F93DF93CF930F92CDB7DEB714
:105920007C01D62E8E010F5F1F4FC80165DF8823D3
:1059300071F0898185DF8981F9DE883541F0C80100
:105940006D2DFBDE8981F701808381E001C080E05D
:105950000F90CF91DF911F910F91FF90EF90DF900B
:1059600008950F931F93DF93CF9300D000D0CDB74E
:10597000DEB78B010E942815CE01019660E1C6DFDB
:10598000882379F1CE01029660E1C0DF882349F1D6
:10599000CE01039660E1BADF882319F1CE010496A7
:1059A00060E1B4DF8823E9F0298130E064E0220F70
:1059B000331F6A95E1F78A81280F311D322F222784
:1059C0008B8190E044E0880F991F4A95E1F74C8164
:1059D000840F911D282B392BF8013183208381E01E
:1059E00001C080E00F900F900F900F90CF91DF914A
:1059F0001F910F910895DF93CF9300D0CDB7DEB7FD
:105A00008AE395E0BE016F5F7F4FABDF882321F013
:105A100089819A810E9443240F900F90CF91DF914A
:105A20000895EF92FF920F931F93DF93CF9300D0CF
:105A3000CDB7DEB78C017B018DED94E00E94281577
:105A4000C8010E942815CE0101966AE05FDF882315
:105A500089F0CE0102966AE059DF882359F08981E6
:105A60002AE0829FC00111242A81280FF701208398
:105A700081E001C080E00F900F90CF91DF911F91E6
:105A80000F91FF90EF9008950F931F93DF93CF93A3
:105A90000F92CDB7DEB78AEF94E08E010F5F1F4FF4
:105AA000B801BFDF882369F184E894E069810E942E
:105AB000F5159981891729F55DDE81E095E0B8013A
:105AC000B0DF8823F1F084E894E069810E94E71553
:105AD00099818917B1F44EDE89E095E0B801A1DF24
:105AE000882379F084E894E069810E94E216998124
:105AF000891739F40E941E1D0E94DB1E1EDA81E008
:105B000004C038DE0E94F71C80E00F90CF91DF9137
:105B10001F910F9108950F931F93DF93CF930F92CF
:105B2000CDB7DEB786EE94E08E010F5F1F4FB80150
:105B300078DF882339F189810E940F1699818917AE
:105B400009F518DE8CEE94E0B8016BDF8823D1F004
:105B500089810E94081699818917A1F40BDE83EFD1
:105B600094E0B8015EDF882369F089810E94011604
:105B70009981891739F40E949F1C0E94DD1EDDD98E
:105B800081E004C080E00E94A11D80E00F90CF91D1
:105B9000DF911F910F910895FF920F931F93DF9351
:105BA000CF930F92CDB7DEB7F82E8B018BEC94E03C
:105BB0000E9428158F2D805D43DE89E241DE8AE355
:105BC0003FDECE0101966AE0A1DE882339F08981AB
:105BD000F81620F0F801808381E001C080E00F908A
:105BE000CF91DF911F910F91FF900895DF93CF9395
:105BF0000F92CDB7DEB785E0BE016F5F7F4FCCDF80
:105C00008823A9F0698180917504681711F481E0F7
:105C10000EC060937504623011F0662329F4698325
:105C200085E190E00E94221481E0809369070F9043
:105C3000CF91DF910895EF92FF921F93DF93CF935F
:105C40000F92CDB7DEB7182F282F30E0C901880F8B
:105C5000991F8F579B4FFC01E590F49023573B4FC2
:105C6000F9018491BE016F5F7F4F96DF882369F051
:105C7000153039F48981853010F0855001C08B5F73
:105C800089838981F701099581E00F90CF91DF9198
:105C90001F91FF90EF900895FC016193CF01642F55
:105CA0000E9484163ECD66E640918D07F5DF62E6E0
:105CB00040918E07F1CF0F931F93DF93CF93CDB712
:105CC000DEB7C054D0400FB6F894DEBF0FBECDBFD4
:105CD0008EE495E00E9428158E010F5F1F4FC801CA
:105CE000E2DF60DDC8010E941C15C05CDF4F0FB60B
:105CF000F894DEBF0FBECDBFCF91DF911F910F9102
:105D000008951F93142F452FC7DF0197612F0E941D
:105D1000841607DD1F9108950F931F93DF93CF9390
:105D2000CDB7DEB7CB54D0400FB6F894DEBF0FBE70
:105D3000CDBFCE0101960E946316F3DC0E9481164E
:105D4000F0DC182F092F84E894E00E941117E82F47
:105D5000F0E0EE0FFF1FE451FF4F65917491812F2A
:105D6000902F0E949C3AA12FB02FFD01019000209E
:105D7000E9F73197EA1BFB0B8E0F9F1FD2DC6CE417
:105D80004091840789DFFC0180918207882311F00C
:105D900086E5819380918C07882311F485E503C003
:105DA000813011F485E4819380919407882311F068
:105DB0008BE4819380918707853059F090E00596B8
:105DC0006AE070E00E941C3A482FCF0162E464DF71
:105DD000FC0180911205882311F086E48193809163
:105DE0007504813011F483E48193CF019ADC5BDF89
:105DF0006DE440918B0750DF40919A0750919B07CB
:105E000069E47FDFCFDCCE0101960E941C15C55BE3
:105E1000DF4F0FB6F894DEBF0FBECDBFCF91DF913D
:105E20001F910F910895AADCA5DC76CFEF92FF9227
:105E30001F93DF93CF930F92CDB7DEB70E94361535
:105E400075DC8983883509F04CC07E010894E11C1B
:105E5000F11C8AEC96E00E942815C701CDDC88234E
:105E600009F443C08981ECDC898160DC182F11546E
:105E700019831F5B80E2E4DC89818A3150F710923C
:105E8000690795E6E92E94E0F92EC701612F70E0CD
:105E90000E94913A009719F08E1925DC1BC08AE701
:105EA000E82E84E0F82EC701612F70E00E94913A3D
:105EB000009719F08E19BFDE0DC0B3E9EB2EB4E0E8
:105EC000FB2EC701612F70E00E94913A009721F0EC
:105ED0008E191CDC882321F48FE095E00E942815A0
:105EE00049DC1ADF2AD8809169070F90CF91DF91A2
:105EF0001F91FF90EF90089580918F0791E089277F
:105F000080938F07882311F48CE301C089E4A7D71D
:105F100081E0089580E086D880E00C941A2683E022
:105F2000809391070AC8582F282F392FACE9B7E082
:105F3000822F851BF9012F5F3F4FE491ED93EE23F4
:105F4000B9F780939207109291070C949D2783E0F4
:105F50009BE19093F3048093F20489E68093F40428
:105F60008DE28093F5048BD880E00E9410268AE1B0
:105F700090E19093800780937F0789E480930D05DB
:105F80008FE0809386048AE2809385040E94A5278F
:105F90008FED96E0C8DFBECF0E94531303D956D7CA
:105FA0008091290390912A03892B11F0F59BF6CF5C
:105FB000F59880E00C94531385E0EECF83E0ECCFAE
:105FC00082E0EACF80E00E941A26FADF83E00E9496
:105FD0001A26F6DF81E00E941A26F2DF81E00E9495
:105FE0001026EEDF80E00E94102682E00E941A2632
:105FF000E7DF80E00E941A26E3DF85E00E941A2690
:10600000DFDF83E00C941A26CF93DF93EC01FE01CF
:106010008491882321F00E94A21F2196F8CFDF915E
:10602000CF910895EF92FF920F931F9381E0809399
:106030006D078DDF9FDB85EE98E10E942815C2DF9A
:1060400086EC97E170DF80E00E941228B7DF85E0E0
:106050000E941228B3DF81E00E941228AFDF82E0A5
:106060000E941228ABDF82EE97E15DDF83E00E94A1
:106070001228A8DF85ED97E156DF84E00E94122800
:10608000A1DF85E298E14FDF82E00E941A2696DFC9
:1060900080E00E94122880E00E941A2685ED98E197
:1060A00042DF8CDF82E398E13EDF8ADF38DF88DF82
:1060B00081E00E94102681E00E9412287FDF80E0AC
:1060C0000E94102683E00E941A2678DF82E00E9458
:1060D000122874DF83E00E94122870DF84E00E949F
:1060E000122880E00E941A2669DF85E00E941228AB
:1060F00082E00E941A2662DF80E00E941A2680E079
:106100000E9412288AEF97E10EDF81E00E9453255A
:1061100053DF82E498E107DF53DF8BE090E1909357
:10612000800780937F074ADF0AE110E11093800720
:1061300000937F0785E598E1F6DE42DF38E6E32E3F
:1061400030E1F32EF0928007E0927F0785E00E9415
:106150001A2681E00E9404282FDF10938007009305
:106160007F0780E00E941A268CE698E1DCDE28DFBB
:10617000F0928007E0927F0784EF60E00E94152094
:1061800085EF60E00E94152086EF60E00E941520F8
:1061900000E010E000933C04C801880F991F880FAD
:1061A000991FFC01ED5AF64EE491E0933D04FC0189
:1061B000EC5AF64EE491E0933E04FC01EB5AF64EA5
:1061C000E491E0933F048A5A964EFC0184918093B7
:1061D000400480EF6CE374E00E94F51F0F5F1F4FD7
:1061E00005361105B9F681EF60E045E60E94D11F42
:1061F00082EF60E04DE00E94D11F8EE598E104DF60
:10620000DBDE84EF61E00E94152085EF61E00E94F3
:1062100015200AE110E11093800700937F078CE7B7
:1062200098E181DECDDEE2D88CE098E17CDEC8DE4C
:106230002AD381E696E0EBD488E590E1909380073D
:1062400080937F07B9DE1093800700937F0780EF6C
:1062500097E169DE82E00E942528B0DE0E943F2897
:10626000AFDE81E00E942528A9DE83E00E94252878
:10627000A5DE0E943F2883E098E155DE8CE00E9475
:10628000E8239CDE83E080936D078CE00E94D0239E
:1062900095DE01E000936D078CE060E01FD68EDE96
:1062A00082ED94E06CE040E050E0F6D687DE88E8CE
:1062B00098E139DE85E080936D0710916E071092AA
:1062C0006E071092CF0478DE10936E0700936D076F
:1062D0008AE998E128DE72DE89EA98E124DE6EDE42
:1062E0008AEB98E120DE6ADE8FEC98E11CDE66DE48
:1062F00011DE8BE198E117DE5FDE0E94351481E04C
:106300001F910F91FF90EF9008958EE58093D10437
:1063100008958091D807E2ECFCE1E80FF11DE491CB
:106320008E2F0895E0918807EF3711F481E00895EA
:10633000EE2311F480E00895EC5FF0E0E453F34EB7
:1063400084910895982F87FF02C0F39A9F7796FF54
:1063500004C081E0809368079F7B892F089580E8BF
:106360009BE19093F3048093F2048BE28093F40416
:106370008DE28093F5040895F59A0895F59A0895AD
:106380008093D1048EE894E018C78093190781E8C0
:1063900094E013D78CEC94E010C788E2F6CF81E943
:1063A00094E00BD71092CB040895D9DFF8DFF59A6B
:1063B0000895F5DF0E941E1D0E94DB1E0E949D278E
:1063C000F59A0895809199078F5F883108F080E0F1
:1063D000809399070C949D27809198078F5F8C3349
:1063E00008F080E0809398070C949D278091970790
:1063F0008F5F8C3308F080E0809397070C949D2783
:1064000084E894E00E94FC150C949D2784E894E0B5
:106410000E94F0150C949D2784E894E06091870415
:106420000E94D716882331F484E894E00E94A616CF
:1064300080938704F59A089584E894E00E94F11609
:106440000C949D2780E00E94A11D0E94F71CA5DFEF
:106450001092F3041092F2040C949D27A0DF86E1C1
:1064600090E0609197070E94221487E190E060918C
:1064700098070E94221488E190E0609199070E9499
:1064800022148BDF0C949D276091CD0780917504B9
:10649000681759F060937504662311F0623021F497
:1064A00085E190E00E94221430CF08950E949F1C45
:1064B0000E94DD1E72DF1092F3041092F2040C941D
:1064C0009D2784E894E00E94DF150E949D2781E0CB
:1064D0000C94242684E894E00E94D7150C949D2700
:1064E00084E894E00E94CF150C949D27AFE5B4E0BA
:1064F000ECE9F7E085E101900D928150E1F7E09140
:10650000F706F0E0E15AFB4F8FE580830895809114
:10651000F706A82FB0E0FD01E456F84FE081EF5FE9
:10652000E7FDE0E2A456B84FEC93E0CF2091CE0710
:106530008CE997E0FC01E20FF11D10820E943F23DD
:106540008093CF0608958093D707E82FF0E0EE0FF1
:10655000FF1FE252F34E259134912093C9063093E8
:10656000CA0680918E0490918F0469EC76E0A901AF
:10657000D0C59091D7079F5F943071F480919A07AE
:1065800080FD0DC0809117078F5F809317078530BE
:1065900028F01092170703C0953008F090E0892F7B
:1065A000D2CF482F8093DB0750E0440F551F440F94
:1065B000551F4B55554E509372064093710680916E
:1065C0008E0490918F0461E776E0A3C58091DB078C
:1065D0008F5F863508F08CE3E4CF8093D807E82FEF
:1065E000F0E0EE0FFF1FE255F34E2591349120931A
:1065F000890630938A0680918E0490918F0469E811
:1066000076E0A90186C58091D8078F5F8A3008F0AF
:1066100080E0E3CF8093CD07E82FF0E0EE0FFF1F7F
:10662000E251F34E259134912093810630938206F6
:1066300080918E0490918F0461E876E0A90169C58C
:106640008091CD078F5F863008F080E0E3CF8093A4
:10665000DA07E82FF0E0EE0FFF1FE655F34E259125
:1066600034912093B9063093BA0680918E049091AC
:106670008F0469EB76E0A9014CC58091DA0791E0BF
:106680008927E5CF8093D507E82FF0E0EE0FFF1FB5
:10669000E655F34E2591349120939106309392065E
:1066A00080918E0490918F0461E976E0A90131C553
:1066B0008091D50791E08927E5CF8093D907E82F0E
:1066C000F0E0EE0FFF1FE856F34E25913491209332
:1066D000C1063093C20680918E0490918F0461ECC4
:1066E00076E0A90116C58091D9078F5F893008F03F
:1066F00080E0E3CF8093D607E82FF0E0EE0FFF1F96
:10670000E851F34E259134912093790630937A061F
:1067100080918E0490918F0469E776E0A901F9C415
:106720008091D6078F5F833008F080E0E3CF8093BD
:10673000D407E82FF0E0EE0FFF1FEA52F34E259149
:1067400034912093B1063093B20680918E049091DB
:106750008F0461EB76E0A901DCC48091D4078F5FE0
:10676000843008F080E0E3CF482F8093D10750E0D9
:10677000440F551F4C59534E5093AA064093A906F7
:1067800080918E0490918F0469EA76E0C2C4809172
:10679000D1078F5F8093D1078A3010F01092D10714
:1067A0008091D107E1CF8093D007E82FF0E0EE0F82
:1067B000FF1FE057F34E259134912093A1063093AB
:1067C000A20680918E0490918F0461EA76E0A9017F
:1067D000A0C48091D0078F5F8093D007843010F0E1
:1067E0001092D0078091D007DECF8093CF07E82F9B
:1067F000F0E0EE0FFF1FE252F34E2591349120930B
:10680000990630939A0680918E0490918F0469E9DD
:1068100076E0A9017EC48091CF0791E08927E5CF7A
:106820008093D207E82FF0E0EE0FFF1FE858F34EF9
:10683000259134912093690630936A0680918E04E5
:1068400090918F0469E676E0A90163C48091D20734
:106850008F5F863008F080E0E3CF8093D307E82F86
:10686000F0E0EE0FFF1FEC57F34E2591349120938B
:1068700061063093620680918E0490918F0461E6E8
:1068800076E0A90146C485E596E060EF7DE14CE73E
:1068900050E03ED680918507A8DF80918907DDDF33
:1068A0008091840780DF809187075EDF80918A076F
:1068B000B7DF809112053BDF80917504ABDE8091DC
:1068C000910741DE1092170780919407DBDE8091DB
:1068D00092078093CE071092F70628DE80918F07EB
:1068E000882321F080919007875B01C08CE359DEFB
:1068F00080918C07FFDE80E0AADE80919507DDDEC7
:1069000011DD6BCE8091D3078F5F863008F080E079
:10691000A4CFEF92FF920F931F938C017B01809184
:10692000810490918204B801A701F3D38091CC0433
:106930009091CD04B801A701ECD31F910F91FF9066
:10694000EF9008950E940E240C94A5274091F7061D
:106950004F5F4093F706642F70E09B012F5F3F4F1E
:106960008091CE0790E02817390724F04F5F4093BD
:10697000CE074150E42FE150443190F09E2F0AC0E1
:10698000292F2150E92FF0E0E456F84F8081803222
:1069900019F4922F9923A1F79F5F9093F70610C0E7
:1069A000EE2319F1E150AE2FB0E0A456B84F8C9110
:1069B0008032D9F411968C918032B9F4E093F706C5
:1069C000E091F706E0939207F0E0E456F84F10826A
:1069D0001092F306B7DFE3DC98CC80E28083A6DD7B
:1069E00085DD8DE58093D1040895FB01E456F84FD1
:1069F0008081882391F3F3CF0E9472240C94A52701
:106A00008091D707823011F4CADCF6CF08956FEF7A
:106A100040E050E041C3CF93DF931092680780912C
:106A2000190790DC982F80931907C4E5DDE101C0B8
:106A30002696FE0184919817D9F7F39B09C0F39825
:106A4000CE010296FC0125913491F901099527C0E8
:106A5000F59B28C0F5982196FE01849173DC95DCA6
:106A6000FE013396C591D4912097C9F0D7FF06C097
:106A70009E012F77822F0E94242611C0CE01C7DFEE
:106A8000909382048093810480916807882339F071
:106A9000CE010496BCDF9093CD048093CC048EE1AC
:106AA0000E945313DF91CF91089580918A049091B1
:106AB0008B04892B19F08AE894E07FD380918907B1
:106AC000833011F482E916C0843011F488EB12C0CF
:106AD00010925D040E94632380918907853011F034
:106AE00089EA08C080918A078350823010F08DEACD
:106AF00001C084EB4ADC8EE10E94531381E0809355
:106B000006030E94D228A2D186DF809129039091AA
:106B10002A03892B11F496DC42DC80911907883214
:106B200081F780918907833051F00E940F1884E12A
:106B30008093B10781E080935D040E94662380E02A
:106B40000E94531381E08093640710920603E4C807
:106B5000CF93DF939091D1049E3539F48091D7077C
:106B6000823019F08FE40CDC4FC0F39B17C0F39810
:106B7000892F90E0805590409C01220F331F280FF1
:106B8000391F220F331F2650334EF90185919491FE
:106B9000FC0109958EE10E94531336C0F59B34C069
:106BA000F598892F90E0805590409C01220F331F6B
:106BB000280F391F220F331F2450334EF9018591BE
:106BC0009491FC0109952091D104822F90E0805589
:106BD0009040FC01EE0FFF1FE80FF91FEE0FFF1FA3
:106BE000E250F34EC591D491822F8F5F8093D104F0
:106BF0008F3508F08FE4C4DB209731F0CE0107DF3A
:106C000090938F0480938E04DF91CF910895FFDEDF
:106C100090938F0480938E0408951F93182F809172
:106C20008A0490918B04892B19F08AE894E0C5D2EC
:106C3000112319F528DE80E5A3DB81E696E0E7DF86
:106C40008EE10E94531381E0809306030E94D228B4
:106C5000FDD07EDF8091290390912A03892B21F4B6
:106C6000CFDE8FE48DDB04C08091D1048F3471F7C7
:106C700081E080936407109206031F9108958DECC4
:106C800096E06FEF4FE554E007D290939204809323
:106C9000910408959091D707923021F41092F7064D
:106CA00025DCEDCF80919107981721F0892F0E9464
:106CB00004282BCB08958AE095E06FEF42ED56E073
:106CC000EBD190939204809391040895F4DFF59AA8
:106CD00008958091DB07C3D0882309F016CB08956F
:106CE0001F9317DB182F80918807181749F087E04A
:106CF00090E0612F0E942214812F0E94C72305DBA0
:106D00001F9108958091DA07882331F0F8940E944A
:106D10004A1C0E943514F9CA08959091D5078091B4
:106D20009407981721F0892F0E941026EECA089523
:106D30001F931091D90780919507181749F0812F5B
:106D40000E94032484E190E0612F0E942214DDDA86
:106D50001F9108959091D60780918C07981721F084
:106D6000892F0E944B25D1CA08959091D407809114
:106D70001205981721F0892F0E942528C6CA089568
:106D80009091D10780918707981721F0892F0E9451
:106D90005624BBCA08959091D00780918407981714
:106DA00021F0892F0E945325B0CA08959091CF07F2
:106DB00080918507981721F0892F0E946024A5CA29
:106DC00008959091D20780918A07981721F0892F12
:106DD0000E9412289ACA08959091D307809189073A
:106DE000981721F0892F0E941A268FCA0895582FCC
:106DF000492F6F5F9C01F90106C08081882339F01B
:106E000031968C32D1F76150C1F75E2F4F2F852F0D
:106E1000942F0895DC018D91FB016F5F7F4FE4910A
:106E20008E1711F080E008958C32A9F781E0089563
:106E3000FC013181305180812AE0829FC001112400
:106E4000380F3C3308F031E0832F089580916707B5
:106E5000882321F00E946B151092670708958C33E8
:106E6000A9F0982F995480918F07882321F0809161
:106E70009007981789F19093900781E080938F078E
:106E8000809195078093830786E00AC080918F07E1
:106E9000882311F11092900710928F078091830739
:106EA0000E9403248EE090E060918F070E942214DC
:106EB0008FE090E0609190070E94221484E190E0BE
:106EC000609195070E94221482E090E06091830710
:106ED0000E94221481E0089580E008950F931F938B
:106EE000CF93DF93082F162FC0E3D2E086EF94E014
:106EF000BE01F5D0892B89F4112321F0D093F7043A
:106F0000C093F60486EF94E0602F40E352E0C4D0D3
:106F1000FC01112311F017821682DF91CF911F918E
:106F20000F910895EF92FF920F931F93DF93CF93EA
:106F3000CDB7DEB7CB54D0400FB6F894DEBF0FBE4E
:106F4000CDBF109267077E010894E11CF11CC701B8
:106F50006AE40E944C158B3408F081C0C7016CE6CE
:106F60007EE158DF882309F47AC0C70162E03FDF81
:106F7000FC018081813409F072C01092640784E0C2
:106F80000E945313C70161E032DF8C0151DF80930F
:106F9000E1060E5F1F4FC8014BDF8093E006C8017A
:106FA000029646DF8093DF06C70169E020DF8C018F
:106FB0003FDF8093E2060E5F1F4FC80139DF8093E9
:106FC000E306C801029634DF8093E40690919007AF
:106FD0008091E106980F9093E10697FF08C0985EB4
:106FE0009093E1068FED96E00E94C01609C098319B
:106FF00038F098519093E1068FED96E00E94F616D6
:107000000E948C1E813011F40E9405178FED96E0CE
:1070100064E874E046E050E096D2009781F0A4E87E
:10702000B4E0EFEDF6E086E001900D928150E1F7DB
:107030000E941E1D0E949F1C81E080936307809127
:107040006307882329F00E94DD1E84E160E006C00A
:1070500080918407833019F084E061E03FDFC55BF5
:10706000DF4F0FB6F894DEBF0FBECDBFCF91DF91DB
:107070001F910F91FF90EF900895809167078823EB
:1070800051F080916407882321F00E945E238823B9
:1070900009F0DCCE47CF0895DC01EAE1F7E030E00B
:1070A00080819181892B71F4B183A0838D919C9112
:1070B000978386839383828381E08483658351876A
:1070C000408705C03F5F3A96363051F735E02AE0F9
:1070D000329F90011124265E384FC9010895AC01FA
:1070E000EAE1F7E09F0180819181009741F08417E8
:1070F000950729F4808591858617970739F03A9688
:1071000087E0E635F80771F720E030E0C90108951F
:107110000895FC01009749F08081918186179707B7
:1071200021F457834683538342830895DC010097FB
:1071300071F0ED91FC91119716968D919C91179796
:10714000918380838AE0FD0111928A95E9F7089581
:10715000AAE1B7E021E08D919C911197892B39F13B
:1071600015968C9115978F3F41F0815015968C9311
:107170001597882311F4CD01D9CF14968C911497CB
:10718000882329F018968D919C91199704C0129626
:107190008D919C911397ED91FC9111979183808330
:1071A00014968C911497822714968C9314971A96A0
:1071B00087E0A635B80779F608950F931F938C01E1
:1071C000FC0180819181B2DFF801118210821F9150
:1071D0000F910895A0E3B0E0EFEEF8E362C1A8E0FC
:1071E0004E010894811C911CF401BA2F1192BA959A
:1071F000E9F729833A834B835C836D837E838F8396
:107200009887CE010996FC011192AA95E9F7A98603
:10721000BA86CB86DC86ED86FE860F87188B2981A1
:107220003A814B815C812DA73EA74FA758AB7901CE
:107230008A018FEF9FEFA0E0B0E0E822F9220A2355
:107240001B231A014424552429853A854B855C85E6
:1072500029A73AA74BA75CA759016A01A822B9221E
:10726000CA22DB223A0188249924C601B501A8016B
:107270009701A3D06DA37EA38FA398A7C401B301E8
:107280009CD069A37AA38BA39CA3C601B501A201DC
:10729000910193D07B018C01C401B3018ED05B01BD
:1072A0006C0189A19AA1ABA1BCA18E0D9F1DA01F4D
:1072B000B11F89A39AA3ABA3BCA32DA13EA14FA14B
:1072C00058A5CA01AA27BB2729A13AA14BA15CA1B5
:1072D000280F391F4A1F5B1F29A33AA34BA35CA3A6
:1072E0002E153F054007510740F480E090E0A1E0F3
:1072F000B0E0A80EB91ECA1EDB1E89A19AA1ABA1DF
:10730000BCA19D01442755272A0D3B1D4C1D5D1D29
:107310002D8F3E8F4F8F58A36C01BB24AA248DA1C3
:107320009EA1AFA1B8A5A070B070A80EB91ECA1ECC
:10733000DB1EA98EBA8ECB8EDC8E9A8C8B8C7C8CCD
:107340009E8D6F8D78A1FE01719688E0DF011D9200
:107350008A95E9F72D8B9E8B6F8B788F2D853E85D7
:107360004F8558896DA57EA58FA598A926D07B014C
:107370008C012D813E814F81588569A57AA58BA509
:107380009CA51BD0E60EF71E081F191F6D897E896C
:107390008F89988D6E0D7F1D801F911F6D8B7E8B49
:1073A0008F8B988FEE892A2D392D482D572D7E2FC2
:1073B0008F89988DE096E2E190C0629FD001739F23
:1073C000F001829FE00DF11D649FE00DF11D929F81
:1073D000F00D839FF00D749FF00D659FF00D9927C0
:1073E000729FB00DE11DF91F639FB00DE11DF91FE4
:1073F000BD01CF0111240895991B79E004C0991FA4
:10740000961708F0961B881F7A95C9F780950895FE
:10741000AA1BBB1B51E107C0AA1FBB1FA617B707BA
:1074200010F0A61BB70B881F991F5A95A9F78095D6
:107430009095BC01CD01089597FB092E07260AD02F
:1074400077FD04D0E5DF06D000201AF47095619531
:107450007F4F0895F6F7909581959F4F0895A1E28B
:107460001A2EAA1BBB1BFD010DC0AA1FBB1FEE1FBE
:10747000FF1FA217B307E407F50720F0A21BB30B09
:10748000E40BF50B661F771F881F991F1A9469F785
:1074900060957095809590959B01AC01BD01CF01E1
:1074A00008952F923F924F925F926F927F928F92A8
:1074B0009F92AF92BF92CF92DF92EF92FF920F9383
:1074C0001F93CF93DF93CDB7DEB7CA1BDB0B0FB68D
:1074D000F894DEBF0FBECDBF09942A88398848884A
:1074E0005F846E847D848C849B84AA84B984C884E0
:1074F000DF80EE80FD800C811B81AA81B981CE0FD7
:10750000D11D0FB6F894DEBF0FBECDBFED010895BB
:10751000FB01DC0102C005900D9241505040D8F7AC
:107520000895FC010590061621F00020D9F7C0014E
:1075300008953197CF010895FB01DC0105900D926C
:107540000020E1F70895FB01DC0104C08D9101905A
:10755000801921F441505040C8F7881B990B0895B9
:10756000FA01CF93FF93EF932230C4F02532B4F4A5
:10757000C22F2C2F332744275527FF93EF936FDF1C
:10758000EF91FF91605D6A330CF0695D6193B90121
:10759000CA01605070408040904059F710828F912E
:1075A0009F91CF9114C0FB019F0142306CF0453296
:1075B0005CF4642F77272CDF805D8A330CF0895DC3
:1075C0008193CB010097A9F71082C90100C0DC01AB
:1075D000FC01672F71917723E1F7329704C07C910A
:1075E0006D9370836291AE17BF07C8F30895F89446
:0275F000FFCFCB
:00000001FF
